:020000040800F2
:10000000B1AA010000000000000000000000000094
:1000100000000000000000000000000000000000E0
:1000200000000000000000000000000000000000D0
:1000300000000000000000000000000000000000C0
:1000400000000000000000000000000000000000B0
:1000500000000000000000000000000000000000A0
:1000600000000000AA50000800000000000000008E
:100070000000000000000000000000000000000080
:100080000000000000000000000000000000000070
:100090000000000000000000000000000000000060
:1000A0000000000000000000000000000000000050
:1000B0000000000000000000000000000000000040
:1000C000F2500008000000000000000000000000E6
:1000D0000000000000000000000000000000000020
:1000E0000000000000000000000000000000000010
:1000F00000000000AC5000080000000000000000FC
:1001000000000000000000000000000000000000EF
:1001100000000000000000000000000000000000DF
:1001200000000000000000000000000000000000CF
:1001300000000000000000000000000000000000BF
:1001400000000000000000000000000000000000AF
:10015000000000000000000094500008737004309C
:10016000170500001305C5FF8545F605637BB5003F
:1001700089816378B500170500001305C5002E9529
:1001800002859302002073A0027D970200009382F3
:1001900062E77390723097A200009382A23A739044
:1001A000C27E73E0C07E97A200009382A23173905A
:1001B000523097110018938161CD178100181301F7
:1001C00061E417C500001305250097050018938505
:1001D00065E3170600181306664D63FAC50083220F
:1001E000050023A0550011059105E3EAC5FE17059A
:1001F00000181305A54B971500189385A57863770C
:10020000B500232005001105E36DB5FE73F0023241
:10021000EF20301A01458145EFA0601401A073E082
:0C0220000232828073F002328280000003
:100240000000000000000000010203040607080986
:100250000000000001000000020000000300000098
:1002600094450008484A000846450008B649000879
:10027000464500084C490008D2460008EC470008F3
:10028000F047000840480008E44800081849000802
:10029000484900084A4500085C45000880450008B8
:1002A0001003520056002D004C0049004E004B0038
:1002B0000000000018034C006F006E006700610032
:1002C0006E0020004E0061006E006F000000000014
:1002D0002E034700440033003200580058005800F5
:1002E0002D0033002E0030002E0030002D0037008E
:1002F0007A0038007800390079006500720000004B
:100300001201000202000040E9288A0100010102F6
:1003100003010000C0C10008A0020008B4020008E8
:10032000D00200083C3F786D6C2076657273696F6F
:100330006E3D22312E30223F3E3C21444F435459E2
:100340005045207461726765742053595354454D6C
:1003500020226764622D7461726765742E64746410
:10036000223E3C7461726765742076657273696FB2
:100370006E3D22312E30223E3C6665617475726599
:10038000206E616D653D226F72672E676E752E67F8
:1003900064622E72697363762E637075223E3C72BE
:1003A0006567206E616D653D227A65726F222062FD
:1003B000697473697A653D22333222207265676EF3
:1003C000756D3D22302220736176652D72657374E0
:1003D0006F72653D227965732220747970653D22C4
:1003E000696E74222067726F75703D2267656E6555
:1003F00072616C222F3E3C726567206E616D653DB7
:10040000227261222062697473697A653D223332F7
:1004100022207265676E756D3D22312220736176F0
:10042000652D726573746F72653D22796573222044
:10043000747970653D22696E74222067726F7570E1
:100440003D2267656E6572616C222F3E3C72656766
:10045000206E616D653D227370222062697473693C
:100460007A653D22333222207265676E756D3D22BA
:10047000322220736176652D726573746F72653DEB
:10048000227965732220747970653D22696E742229
:100490002067726F75703D2267656E6572616C22B0
:1004A0002F3E3C726567206E616D653D226770224C
:1004B0002062697473697A653D2233322220726545
:1004C000676E756D3D22332220736176652D7265EE
:1004D00073746F72653D227965732220747970653B
:1004E0003D22696E74222067726F75703D226765C8
:1004F0006E6572616C222F3E3C726567206E616D85
:10050000653D227470222062697473697A653D22A8
:10051000333222207265676E756D3D22342220735E
:100520006176652D726573746F72653D22796573AE
:100530002220747970653D22696E74222067726F83
:1005400075703D2267656E6572616C222F3E3C724C
:100550006567206E616D653D22743022206269748A
:1005600073697A653D22333222207265676E756D3C
:100570003D22352220736176652D726573746F722A
:10058000653D227965732220747970653D22696E1C
:1005900074222067726F75703D2267656E657261A7
:1005A0006C222F3E3C726567206E616D653D227442
:1005B00031222062697473697A653D2233322220C8
:1005C0007265676E756D3D22362220736176652DEA
:1005D000726573746F72653D227965732220747938
:1005E00070653D22696E74222067726F75703D22BE
:1005F00067656E6572616C222F3E3C726567206E86
:10060000616D653D227432222062697473697A6576
:100610003D22333222207265676E756D3D2237228E
:1006200020736176652D726573746F72653D2279F2
:1006300065732220747970653D22696E742220678B
:10064000726F75703D2267656E6572616C222F3E18
:100650003C726567206E616D653D22667022206286
:10066000697473697A653D22333222207265676E40
:10067000756D3D22382220736176652D7265737425
:100680006F72653D227965732220747970653D2211
:10069000696E74222067726F75703D2267656E65A2
:1006A00072616C222F3E3C726567206E616D653D04
:1006B000227331222062697473697A653D22333274
:1006C00022207265676E756D3D2239222073617636
:1006D000652D726573746F72653D22796573222092
:1006E000747970653D22696E74222067726F75702F
:1006F0003D2267656E6572616C222F3E3C726567B4
:10070000206E616D653D22613022206269747369DB
:100710007A653D22333222207265676E756D3D2207
:1007200031302220736176652D726573746F726546
:100730003D227965732220747970653D22696E745B
:10074000222067726F75703D2267656E6572616CFD
:10075000222F3E3C726567206E616D653D226131DE
:10076000222062697473697A653D223332222072D5
:1007700065676E756D3D2231312220736176652D7E
:10078000726573746F72653D227965732220747986
:1007900070653D22696E74222067726F75703D220C
:1007A00067656E6572616C222F3E3C726567206ED4
:1007B000616D653D226132222062697473697A65D8
:1007C0003D22333222207265676E756D3D223132D3
:1007D0002220736176652D726573746F72653D2298
:1007E0007965732220747970653D22696E742220C8
:1007F00067726F75703D2267656E6572616C222F3E
:100800003E3C726567206E616D653D22613322203A
:1008100062697473697A653D22333222207265679A
:100820006E756D3D2231332220736176652D7265C0
:1008300073746F72653D22796573222074797065D7
:100840003D22696E74222067726F75703D22676564
:100850006E6572616C222F3E3C726567206E616D21
:10086000653D226134222062697473697A653D2294
:10087000333222207265676E756D3D22313422203D
:10088000736176652D726573746F72653D2279654B
:10089000732220747970653D22696E74222067721C
:1008A0006F75703D2267656E6572616C222F3E3CEC
:1008B000726567206E616D653D2261352220626937
:1008C0007473697A653D22333222207265676E75D2
:1008D0006D3D2231352220736176652D726573740A
:1008E0006F72653D227965732220747970653D22AF
:1008F000696E74222067726F75703D2267656E6540
:1009000072616C222F3E3C726567206E616D653DA1
:10091000226136222062697473697A653D2233321E
:1009200022207265676E756D3D223136222073611B
:1009300076652D726573746F72653D2279657322D9
:1009400020747970653D22696E74222067726F751C
:10095000703D2267656E6572616C222F3E3C726548
:1009600067206E616D653D22613722206269747374
:10097000697A653D22333222207265676E756D3D5E
:100980002231372220736176652D726573746F7220
:10099000653D227965732220747970653D22696E08
:1009A00074222067726F75703D2267656E65726193
:1009B0006C222F3E3C726567206E616D653D22732F
:1009C00032222062697473697A653D2233322220B3
:1009D0007265676E756D3D223138222073617665D0
:1009E0002D726573746F72653D2279657322207470
:1009F0007970653D22696E74222067726F75703D53
:100A00002267656E6572616C222F3E3C72656720BD
:100A10006E616D653D227333222062697473697A59
:100A2000653D22333222207265676E756D3D22313D
:100A3000392220736176652D726573746F72653D1E
:100A4000227965732220747970653D22696E742263
:100A50002067726F75703D2267656E6572616C22EA
:100A60002F3E3C726567206E616D653D22733422B6
:100A70002062697473697A653D223332222072657F
:100A8000676E756D3D2232302220736176652D725E
:100A90006573746F72653D22796573222074797075
:100AA000653D22696E74222067726F75703D226702
:100AB000656E6572616C222F3E3C726567206E61C7
:100AC0006D653D227335222062697473697A653DD4
:100AD00022333222207265676E756D3D22323122DB
:100AE00020736176652D726573746F72653D22792E
:100AF00065732220747970653D22696E74222067C7
:100B0000726F75703D2267656E6572616C222F3E53
:100B10003C726567206E616D653D227336222062EE
:100B2000697473697A653D22333222207265676E7B
:100B3000756D3D2232322220736176652D726573A8
:100B4000746F72653D227965732220747970653DFA
:100B500022696E74222067726F75703D2267656E20
:100B60006572616C222F3E3C726567206E616D6517
:100B70003D227337222062697473697A653D22339E
:100B80003222207265676E756D3D223233222073EA
:100B90006176652D726573746F72653D2279657338
:100BA0002220747970653D22696E74222067726F0D
:100BB00075703D2267656E6572616C222F3E3C72D6
:100BC0006567206E616D653D22733822206269740D
:100BD00073697A653D22333222207265676E756DC6
:100BE0003D2232342220736176652D726573746FF5
:100BF00072653D227965732220747970653D2269A2
:100C00006E74222067726F75703D2267656E657223
:100C1000616C222F3E3C726567206E616D653D22DE
:100C20007339222062697473697A653D22333222F6
:100C3000207265676E756D3D2232352220736176B4
:100C4000652D726573746F72653D2279657322201C
:100C5000747970653D22696E74222067726F7570B9
:100C60003D2267656E6572616C222F3E3C7265673E
:100C7000206E616D653D227331302220626974738C
:100C8000697A653D22333222207265676E756D3D4B
:100C90002232362220736176652D726573746F720D
:100CA000653D227965732220747970653D22696EF5
:100CB00074222067726F75703D2267656E65726180
:100CC0006C222F3E3C726567206E616D653D22731C
:100CD0003131222062697473697A653D2233322290
:100CE000207265676E756D3D223237222073617602
:100CF000652D726573746F72653D2279657322206C
:100D0000747970653D22696E74222067726F757008
:100D10003D2267656E6572616C222F3E3C7265678D
:100D2000206E616D653D227433222062697473699F
:100D30007A653D22333222207265676E756D3D22E1
:100D400032382220736176652D726573746F726517
:100D50003D227965732220747970653D22696E7435
:100D6000222067726F75703D2267656E6572616CD7
:100D7000222F3E3C726567206E616D653D227434A2
:100D8000222062697473697A653D223332222072AF
:100D900065676E756D3D2232392220736176652D4F
:100DA000726573746F72653D227965732220747960
:100DB00070653D22696E74222067726F75703D22E6
:100DC00067656E6572616C222F3E3C726567206EAE
:100DD000616D653D227435222062697473697A659C
:100DE0003D22333222207265676E756D3D223330AD
:100DF0002220736176652D726573746F72653D2272
:100E00007965732220747970653D22696E742220A1
:100E100067726F75703D2267656E6572616C222F17
:100E20003E3C726567206E616D653D2274362220FE
:100E300062697473697A653D223332222072656774
:100E40006E756D3D2233312220736176652D72659A
:100E500073746F72653D22796573222074797065B1
:100E60003D22696E74222067726F75703D2267653E
:100E70006E6572616C222F3E3C726567206E616DFB
:100E8000653D227063222062697473697A653D2230
:100E9000333222207265676E756D3D223332222017
:100EA000736176652D726573746F72653D22796525
:100EB000732220747970653D22696E7422206772F6
:100EC0006F75703D2267656E6572616C222F3E3CC6
:100ED0002F666561747572653E3C666561747572F6
:100EE00065206E616D653D226F72672E676E752E8F
:100EF0006764622E72697363762E637372223E3C5E
:100F0000726567206E616D653D226D7374617475E5
:100F100073222062697473697A653D22333222201C
:100F20007265676E756D3D223833332220736176AA
:100F3000652D726573746F72653D226E6F22207429
:100F40007970653D22696E74222067726F75703DFD
:100F500022637372222F3E3C726567206E616D655D
:100F60003D226D697361222062697473697A653DFF
:100F700022333222207265676E756D3D223833341C
:100F80002220736176652D726573746F72653D22E0
:100F90006E6F2220747970653D22696E742220671D
:100FA000726F75703D22637372222F3E3C726567CB
:100FB000206E616D653D226D6965222062697473E2
:100FC000697A653D22333222207265676E756D3D08
:100FD000223833372220736176652D726573746F02
:100FE00072653D226E6F2220747970653D22696EB4
:100FF00074222067726F75703D22637372222F3ED8
:101000003C726567206E616D653D226D7476656327
:10101000222062697473697A653D2233322220721C
:1010200065676E756D3D22383338222073617665B1
:101030002D726573746F72653D226E6F2220747914
:1010400070653D22696E74222067726F75703D2253
:10105000637372222F3E3C726567206E616D653D41
:10106000226D636F756E746572656E22206269749D
:1010700073697A653D22333222207265676E756D21
:101080003D223833392220736176652D7265737481
:101090006F72653D226E6F2220747970653D226902
:1010A0006E74222067726F75703D22637372222FF7
:1010B0003E3C726567206E616D653D226D636F75A4
:1010C0006E74696E686962697422206269747369FA
:1010D0007A653D22333222207265676E756D3D223E
:1010E0003836352220736176652D726573746F72A0
:1010F000653D226E6F2220747970653D22696E74A1
:10110000222067726F75703D22637372222F3E3CFE
:10111000726567206E616D653D226D7363726174E7
:101120006368222062697473697A653D22333222D2
:10113000207265676E756D3D2238393722207361E4
:1011400076652D726573746F72653D226E6F222015
:10115000747970653D22696E74222067726F7570B4
:101160003D22637372222F3E3C726567206E616D73
:10117000653D226D657063222062697473697A65CA
:101180003D22333222207265676E756D3D223839FB
:10119000382220736176652D726573746F72653DB8
:1011A000226E6F2220747970653D22696E74222050
:1011B00067726F75703D22637372222F3E3C7265B9
:1011C00067206E616D653D226D63617573652220D8
:1011D00062697473697A653D2233322220726567D1
:1011E0006E756D3D223839392220736176652D7216
:1011F0006573746F72653D226E6F2220747970651D
:101200003D22696E74222067726F75703D22637390
:1012100072222F3E3C726567206E616D653D226DC6
:101220007476616C222062697473697A653D223339
:101230003222207265676E756D3D22393030222072
:10124000736176652D726573746F72653D226E6F82
:101250002220747970653D22696E74222067726F56
:1012600075703D22637372222F3E3C726567206E5B
:10127000616D653D226D6970222062697473697ABF
:10128000653D22333222207265676E756D3D2239CD
:1012900030312220736176652D726573746F7265CB
:1012A0003D226E6F2220747970653D22696E742232
:1012B0002067726F75703D22637372222F3E3C72FD
:1012C0006567206E616D653D227473656C6563743E
:1012D000222062697473697A653D2233322220725A
:1012E00065676E756D3D223230313722207361762D
:1012F000652D726573746F72653D226E6F22207466
:101300007970653D22696E74222067726F75703D39
:1013100022637372222F3E3C726567206E616D6599
:101320003D22746461746131222062697473697A48
:10133000653D22333222207265676E756D3D223223
:101340003031382220736176652D726573746F7247
:10135000653D226E6F2220747970653D22696E743E
:10136000222067726F75703D22637372222F3E3C9C
:10137000726567206E616D653D22746461746132CF
:10138000222062697473697A653D223332222072A9
:1013900065676E756D3D223230313922207361767A
:1013A000652D726573746F72653D226E6F222074B5
:1013B0007970653D22696E74222067726F75703D89
:1013C00022637372222F3E3C726567206E616D65E9
:1013D0003D22746461746133222062697473697A96
:1013E000653D22333222207265676E756D3D223273
:1013F0003032302220736176652D726573746F729E
:10140000653D226E6F2220747970653D22696E748D
:10141000222067726F75703D22637372222F3E3CEB
:10142000726567206E616D653D2264637372222070
:1014300062697473697A653D22333222207265676E
:101440006E756D3D22323033332220736176652D07
:10145000726573746F72653D226E6F2220747970AD
:10146000653D22696E74222067726F75703D22633C
:101470007372222F3E3C726567206E616D653D225E
:10148000647063222062697473697A653D22333225
:1014900022207265676E756D3D2232303334222012
:1014A000736176652D726573746F72653D226E6F20
:1014B0002220747970653D22696E74222067726FF4
:1014C00075703D22637372222F3E3C726567206EF9
:1014D000616D653D2264736372617463682220628A
:1014E000697473697A653D22333222207265676EB2
:1014F000756D3D22323033352220736176652D7251
:101500006573746F72653D226E6F22207479706509
:101510003D22696E74222067726F75703D2263737D
:1015200072222F3E3C726567206E616D653D226DB3
:101530006379636C65222062697473697A653D2200
:10154000333222207265676E756D3D223238383134
:101550002220736176652D726573746F72653D220A
:101560006E6F2220747970653D22696E7422206747
:10157000726F75703D22637372222F3E3C726567F5
:10158000206E616D653D226D696E737472657422A3
:101590002062697473697A653D2233322220726554
:1015A000676E756D3D22323838332220736176655F
:1015B0002D726573746F72653D226E6F222074798F
:1015C00070653D22696E74222067726F75703D22CE
:1015D000637372222F3E3C726567206E616D653DBC
:1015E000226D6379636C6568222062697473697A1D
:1015F000653D22333222207265676E756D3D223360
:101600003030392220736176652D726573746F7284
:10161000653D226E6F2220747970653D22696E747B
:10162000222067726F75703D22637372222F3E3CD9
:10163000726567206E616D653D226D696E737472AF
:10164000657468222062697473697A653D22333259
:1016500022207265676E756D3D2233303131222054
:10166000736176652D726573746F72653D226E6F5E
:101670002220747970653D22696E74222067726F32
:1016800075703D22637372222F3E3C726567206E37
:10169000616D653D226379636C65222062697473B4
:1016A000697A653D22333222207265676E756D3D21
:1016B00022333133372220736176652D726573745E
:1016C0006F72653D226E6F2220747970653D2269CC
:1016D0006E74222067726F75703D22637372222FC1
:1016E0003E3C726567206E616D653D2274696D6573
:1016F000222062697473697A653D22333222207236
:1017000065676E756D3D2233313338222073617603
:10171000652D726573746F72653D226E6F22207441
:101720007970653D22696E74222067726F75703D15
:1017300022637372222F3E3C726567206E616D6575
:101740003D22696E737472657422206269747369D4
:101750007A653D22333222207265676E756D3D22B7
:10176000333133392220736176652D726573746F5E
:1017700072653D226E6F2220747970653D22696E1C
:1017800074222067726F75703D22637372222F3E40
:101790003C726567206E616D653D226379636C659F
:1017A00068222062697473697A653D22333222208F
:1017B0007265676E756D3D22333236352220736156
:1017C00076652D726573746F72653D226E6F22208F
:1017D000747970653D22696E74222067726F75702E
:1017E0003D22637372222F3E3C726567206E616DED
:1017F000653D2274696D6568222062697473697A37
:10180000653D22333222207265676E756D3D22334D
:101810003236362220736176652D726573746F726D
:10182000653D226E6F2220747970653D22696E7469
:10183000222067726F75703D22637372222F3E3CC7
:10184000726567206E616D653D22696E73747265A5
:101850007468222062697473697A653D223332228A
:10186000207265676E756D3D2233323637222073E4
:101870006176652D726573746F72653D226E6F229D
:1018800020747970653D22696E74222067726F75CD
:10189000703D22637372222F3E3C726567206E6139
:1018A0006D653D226D76656E646F7269642220629B
:1018B000697473697A653D22333222207265676EDE
:1018C000756D3D22333932322220736176652D7277
:1018D0006573746F72653D226E6F22207479706536
:1018E0003D22696E74222067726F75703D226373AA
:1018F00072222F3E3C726567206E616D653D226DE0
:10190000617263686964222062697473697A653DF3
:1019100022333222207265676E756D3D2233393273
:10192000332220736176652D726573746F72653D25
:10193000226E6F2220747970653D22696E742220B8
:1019400067726F75703D22637372222F3E3C726521
:1019500067206E616D653D226D696D70696422203E
:1019600062697473697A653D223332222072656739
:101970006E756D3D22333932342220736176652DC8
:10198000726573746F72653D226E6F222074797078
:10199000653D22696E74222067726F75703D226307
:1019A0007372222F3E3C726567206E616D653D2229
:1019B0006D686172746964222062697473697A6502
:1019C0003D22333222207265676E756D3D223339B8
:1019D00032352220736176652D726573746F72657E
:1019E0003D226E6F2220747970653D22696E7422EB
:1019F0002067726F75703D22637372222F3E3C72B6
:101A00006567206E616D653D226D7476742220627B
:101A1000697473697A653D22333222207265676E7C
:101A2000756D3D223834302220736176652D7265E4
:101A300073746F72653D226E6F2220747970653DFC
:101A400022696E74222067726F75703D2263737213
:101A5000222F3E3C726567206E616D653D226D6987
:101A60006E74737461747573222062697473697A19
:101A7000653D22333222207265676E756D3D2239D5
:101A800030332220736176652D726573746F7265D1
:101A90003D226E6F2220747970653D22696E74223A
:101AA0002067726F75703D22637372222F3E3C7205
:101AB0006567206E616D653D226D7363726174634D
:101AC00068637377222062697473697A653D223393
:101AD0003222207265676E756D3D223930352220C5
:101AE000736176652D726573746F72653D226E6FDA
:101AF0002220747970653D22696E74222067726FAE
:101B000075703D22637372222F3E3C726567206EB2
:101B1000616D653D226D7363726174636863737791
:101B20006C222062697473697A653D223332222007
:101B30007265676E756D3D2239303622207361768D
:101B4000652D726573746F72653D226E6F2220740D
:101B50007970653D22696E74222067726F75703DE1
:101B600022637372222F3E3C726567206E616D6541
:101B70003D226D6E766563222062697473697A65B1
:101B80003D22333222207265676E756D3D22323000
:101B900035322220736176652D726573746F7265BC
:101BA0003D226E6F2220747970653D22696E742229
:101BB0002067726F75703D22637372222F3E3C72F4
:101BC0006567206E616D653D226D7375626D2220C3
:101BD00062697473697A653D2233322220726567C7
:101BE0006E756D3D22323035332220736176652D5E
:101BF000726573746F72653D226E6F222074797006
:101C0000653D22696E74222067726F75703D226394
:101C10007372222F3E3C726567206E616D653D22B6
:101C20006D6D6973635F63746C222062697473699C
:101C30007A653D22333222207265676E756D3D22D2
:101C4000323036352220736176652D726573746F7C
:101C500072653D226E6F2220747970653D22696E37
:101C600074222067726F75703D22637372222F3E5B
:101C70003C726567206E616D653D226D73617665AE
:101C8000737461747573222062697473697A653D37
:101C900022333222207265676E756D3D22323037F5
:101CA000312220736176652D726573746F72653DA4
:101CB000226E6F2220747970653D22696E74222035
:101CC00067726F75703D22637372222F3E3C72659E
:101CD00067206E616D653D226D7361766565706329
:101CE00031222062697473697A653D223332222081
:101CF0007265676E756D3D22323037322220736116
:101D000076652D726573746F72653D226E6F222049
:101D1000747970653D22696E74222067726F7570E8
:101D20003D22637372222F3E3C726567206E616DA7
:101D3000653D226D7361766563617573653122203F
:101D400062697473697A653D223332222072656755
:101D50006E756D3D22323037332220736176652DEA
:101D6000726573746F72653D226E6F222074797094
:101D7000653D22696E74222067726F75703D226323
:101D80007372222F3E3C726567206E616D653D2245
:101D90006D73617665657063322220626974736960
:101DA0007A653D22333222207265676E756D3D2261
:101DB000323037342220736176652D726573746F0B
:101DC00072653D226E6F2220747970653D22696EC6
:101DD00074222067726F75703D22637372222F3EEA
:101DE0003C726567206E616D653D226D736176653D
:101DF000636175736532222062697473697A653D27
:101E000022333222207265676E756D3D2232303783
:101E1000352220736176652D726573746F72653D2E
:101E2000226E6F2220747970653D22696E742220C3
:101E300067726F75703D22637372222F3E3C72652C
:101E400067206E616D653D226D747674322220626A
:101E5000697473697A653D22333222207265676E38
:101E6000756D3D22323039332220736176652D72D3
:101E70006573746F72653D226E6F22207479706590
:101E80003D22696E74222067726F75703D22637304
:101E900072222F3E3C726567206E616D653D227334
:101EA0006C65657076616C75652220626974736912
:101EB0007A653D22333222207265676E756D3D2250
:101EC000323133302220736176652D726573746F01
:101ED00072653D226E6F2220747970653D22696EB5
:101EE00074222067726F75703D22637372222F3ED9
:101EF0003C726567206E616D653D2274786576740D
:101F0000222062697473697A653D2233322220721D
:101F100065676E756D3D22323133312220736176F3
:101F2000652D726573746F72653D226E6F22207429
:101F30007970653D22696E74222067726F75703DFD
:101F400022637372222F3E3C726567206E616D655D
:101F50003D22776665222062697473697A653D2245
:101F6000333222207265676E756D3D22323132390F
:101F70002220736176652D726573746F72653D22E0
:101F80006E6F2220747970653D22696E742220671D
:101F9000726F75703D22637372222F3E3C2F66650F
:101FA00061747572653E3C66656174757265206E1C
:101FB000616D653D226F72672E676E752E67646274
:101FC0002E72697363762E7669727475616C223E27
:101FD0003C726567206E616D653D22707269762284
:101FE0002062697473697A653D22382220726567C0
:101FF0006E756D3D22343136312220736176652D48
:10200000726573746F72653D226E6F2220747970F1
:10201000653D22696E74222067726F75703D22677C
:10202000656E6572616C222F3E3C2F66656174752A
:1020300072653E3C2F7461726765743E000000005B
:10204000D25D0008FA5D0008F45D0008FA5D000842
:10205000D25D0008FA5D0008F45D0008FA5D000832
:10206000D25D0008FA5D0008F45D0008FA5D000822
:10207000FA5D0008FA5D0008FA5D0008FA5D0008E4
:10208000D25D0008FA5D0008F45D0008FA5D000802
:10209000D25D0008FA5D0008F45D0008FA5D0008F2
:1020A000D25D0008FA5D0008F45D0008005E0008DB
:1020B000845E00082C5E0008845E0008125E000842
:1020C000845E0008465E0008845E0008125E000818
:1020D000845E0008465E0008845E0008845E000896
:1020E000845E0008845E0008845E0008005E0008CC
:1020F000845E0008605E0008845E0008125E0008CE
:10210000845E0008725E0008845E0008125E0008AB
:10211000845E0008725E00086E6F206572726F72D6
:10212000000000006162733A3020286E6F6E6529EE
:10213000000000006162733A3120286275737929CA
:10214000000000006162733A3220286E6F742073C1
:102150007570706F72746564290000006162733A73
:10216000332028657863657074696F6E29000000FC
:102170006162733A34202868616C742F72657375DC
:102180006D6529006162733A3520286275732900F4
:102190006162733A3620284649584D4529000000AF
:1021A0006162733A3720286F7468657229000000F5
:1021B0004744333256463130330000002530327800
:1021C00000000000D4A1000836A3000836A30008D0
:1021D00036A3000836A3000836A3000836A300087B
:1021E00036A3000836A3000836A3000836A300086B
:1021F00036A3000836A3000836A3000836A300085B
:1022000036A3000836A3000836A3000836A300084A
:1022100036A3000836A3000836A3000836A300083A
:1022200036A3000836A3000836A3000836A300082A
:1022300036A3000836A3000836A3000836A300081A
:1022400036A3000836A3000836A3000836A300080A
:1022500036A3000836A3000836A3000836A30008FA
:1022600036A3000836A3000836A3000836A30008EA
:1022700036A3000836A3000836A3000836A30008DA
:1022800036A3000836A3000836A3000836A30008CA
:1022900036A3000836A3000836A3000836A30008BA
:1022A00036A3000836A3000836A3000836A30008AA
:1022B00036A3000836A3000836A3000836A300089A
:1022C00036A3000836A3000836A3000836A300088A
:1022D00036A3000836A3000836A3000836A300087A
:1022E00036A3000836A3000836A3000836A300086A
:1022F00036A3000836A3000836A3000836A300085A
:1023000036A3000836A3000836A3000836A3000849
:1023100036A3000836A3000836A3000836A3000839
:1023200036A3000836A3000836A3000836A3000829
:1023300036A3000836A3000836A3000836A3000819
:1023400036A3000836A3000836A3000836A3000809
:1023500036A3000836A3000836A3000836A30008F9
:1023600036A3000836A3000836A3000836A30008E9
:1023700036A3000836A3000836A3000836A30008D9
:1023800036A3000836A3000836A3000836A30008C9
:1023900036A3000836A3000836A3000836A30008B9
:1023A000009F000836A3000836A3000836A30008E3
:1023B00036A3000836A3000836A3000836A3000899
:1023C00036A3000836A3000836A3000836A3000889
:1023D00036A3000836A3000836A3000848A000086A
:1023E00036A3000836A3000836A3000836A3000869
:1023F00036A3000836A3000886A0000836A300080C
:1024000036A3000836A3000836A3000836A3000848
:1024100036A3000836A3000836A30008CCA00008A5
:1024200036A3000836A3000836A3000836A3000828
:1024300036A3000836A3000836A3000836A3000818
:1024400036A3000836A3000836A3000836A3000808
:1024500036A3000836A3000836A3000836A30008F8
:1024600036A3000836A3000836A3000836A30008E8
:1024700036A3000836A3000836A30008149F0008FE
:1024800036A3000836A30008349F000836A30008CE
:1024900036A3000836A30008C6A1000836A300082A
:1024A000EEA1000836A3000804A2000836A3000825
:1024B0001AA2000836A3000830A2000836A30008BC
:1024C00046A2000836A300085CA2000836A3000854
:1024D00072A2000836A3000888A2000836A30008EC
:1024E0009EA2000836A30008B4A2000836A3000884
:1024F000CAA2000836A30008E0A2000836A300081C
:10250000F6A2000836A300080CA3000836A30008B2
:1025100022A3000836A30008E09F000825780000E9
:102520005153746172744E6F41636B4D6F646500FB
:102530005A25782C25782C25780000007153757069
:10254000706F727465643A0071586665723A6665B8
:102550006174757265733A726561643A7461726729
:1025600065742E786D6C3A0071586665723A6D65C7
:102570006D6F72792D6D61703A726561643A3A00DF
:102580007152636D642C0000726573657400000005
:1025900068616C740000000073686F772065727268
:1025A0006F72000052562D4C494E4B204552524FEF
:1025B000523A2025732C20403078253038780D0A87
:1025C000000000003A2820756E737570706F727489
:1025D0006564206D6F6E69746F7220636F6D6D61DD
:1025E0006E64210A000000005061636B65745369DA
:1025F0007A653D3430353B5153746172744E6F418E
:10260000636B4D6F64652B3B71586665723A666506
:102610006174757265733A726561642B3B715866BB
:1026200065723A6D656D6F72792D6D61703A726584
:1026300061642B3B7377627265616B2B3B687762D9
:102640007265616B2B0000005330320072616D00C7
:10265000666C6173680000006C3C6D656D6F72792B
:102660002D6D61703E0000003C6D656D6F727920CC
:10267000747970653D222573222073746172743DF4
:10268000223078257822206C656E6774683D223090
:1026900078257822000000003E3C70726F706572F1
:1026A0007479206E616D653D22626C6F636B736936
:1026B0007A65223E307825783C2F70726F70657293
:1026C00074793E3C2F6D656D6F72793E000000009D
:1026D0002F3E00003C2F6D656D6F72792D6D61701E
:1026E0003E00000076466C61736845726173653A1E
:1026F0000000000076466C61736857726974653A31
:102700000000000076466C617368446F6E650000DF
:10271000764D7573745265706C79456D707479007F
:102720007A25782C25782C25780000000A52562D21
:102730004C494E4B204552524F523A207468652006
:10274000746172676574206973206E6F7420636FA3
:102750006E6E6563746564210A0000000A52562D8E
:102760004C494E4B204552524F523A2074686520D6
:10277000746172676574206973206E6F742073755D
:1027800070706F727465642C207570677261646517
:102790002052562D4C494E4B206669726D776172FE
:1027A00065210A000A52562D4C494E4B2045525283
:1027B0004F523A20736F6D657468696E6720777247
:1027C0006F6E672077697468206465627567206D35
:1027D0006F64756C65210A000A52562D4C494E4BA8
:1027E000204552524F523A207468652074617267D6
:1027F000657420756E6465722070726F74656374A1
:102800006564212064697361626C652070726F7405
:10281000656374696F6E207468656E2074727920C8
:10282000616761696E2E0A000A52562D4C494E4B63
:10283000204552524F523A20756E6B6E6F776E2064
:102840006572726F72210A0052562D4C494E4B2010
:1028500076302E323A2000004C6F6E67616E204E4B
:10286000616E6F002C20636F6E6669676564206619
:102870006F7220002066616D696C792E0A0000007D
:102880005430320054303500543035776174636809
:102890003A25783B0000000054303572776174634C
:1028A000683A25783B0000005430356177617463E5
:1028B000683A25783B0000005430356877627265CD
:1028C000616B3A3B000000005430357377627265EB
:1028D000616B3A3B00000000452530327800000073
:1028E0004F4B00000001020203030303040404042D
:1028F000040404040505050505050505050505058C
:10290000050505050606060606060606060606066B
:102910000606060606060606060606060606060657
:10292000060606060707070707070707070707073B
:102930000707070707070707070707070707070727
:102940000707070707070707070707070707070717
:102950000707070707070707070707070707070707
:1029600007070707080808080808080808080808EB
:1029700008080808080808080808080808080808D7
:1029800008080808080808080808080808080808C7
:1029900008080808080808080808080808080808B7
:1029A00008080808080808080808080808080808A7
:1029B0000808080808080808080808080808080897
:1029C0000808080808080808080808080808080887
:1029D0000808080808080808080808080808080877
:1029E00008080808232D302B20000000686C4C00DC
:1029F0006566674546470000303132333435363737
:102A000038394142434445460000000030313233FA
:102A1000343536373839616263646566000000001A
:102A2000412D46612D6638393031323334353637F1
:102A30005D0000002B2D00003030000078580000B1
:102A40000000000000000000000000000000000086
:102A50000000000000000000000000000000000076
:102A60000000000000000000000000000000000066
:102A70000000000000000000000000000000000056
:102A80000000000000000000000000000000000046
:102A90000000000000000000000000000000000036
:102AA00043000000504F5349580000002E00000022
:102AB000002020202020202020202828282828200E
:102AC0002020202020202020202020202020202006
:102AD000208810101010101010101010101010106E
:102AE000100404040404040404040410101010105E
:102AF0001010414141414141010101010101010128
:102B00000101010101010101010101011010101079
:102B100010104242424242420202020202020202F9
:102B2000020202020202020202020202101010104D
:102B30002000000000000000000000000000000075
:102B40000000000000000000000000000000000085
:102B50000000000000000000000000000000000075
:102B60000000000000000000000000000000000065
:102B70000000000000000000000000000000000055
:102B80000000000000000000000000000000000045
:102B90000000000000000000000000000000000035
:102BA0000000000000000000000000000000000025
:102BB0000000411106C68124130570058920952A5D
:102BC000B240410182808280B707002003A7876856
:102BD0003A95B727002093870798636EF500B7876B
:102BE00000209387078063EAA700B707002023A48B
:102BF000A7683A8582807D57EDBF7D57DDBFB70757
:102C000000D223800700A38507001205B71700D262
:102C10003E9563F6A70023A00700C107DDBF8280B1
:102C20000A05B71700D285073E9585472300F500B2
:102C300082800A05B71700D28D073E952300B500A4
:102C400082800A05B71700D28D073E95034505001F
:102C50008280B70700D22380A7008280B70700D206
:102C600003C507008280411106C622C406051374FD
:102C7000F50FED371375150E7988418DD93FB240A8
:102C8000224441018280411106C6C93F05813D8928
:102C9000B24041018280411106C622C426C24AC008
:102CA0002A892E84CD37AA84914763F3A7009144E3
:102CB000A147858F3314F4001374F40F4A855137FC
:102CC000B315950093F5F50FB3D5954093F5F50F32
:102CD000C18D4A85B93FB240224492440249410124
:102CE0008280411106C622C426C24AC02A892E8487
:102CF000593F8D4763FAA70001442285B240224420
:102D00009244024941018280AA8412041374F40F90
:102D10004A85053FA145B3849540B355954093F549
:102D2000F50FB395950093F5F50FC18D4A851137D1
:102D3000E9B7F327503093F707FC93E73700739018
:102D400057308280371702401C43C166D58F1CC3A1
:102D5000814785073717024018439316E70063C67B
:102D6000060041677D17E396E7FEB71702409C43D4
:102D70001397E7006343070001A0B7170240D84349
:102D8000D8C3D843D8C3D84313670740D8C3D84360
:102D9000B706C4DFFD16758FD8C3D843B7061D200C
:102DA000558FD8C3D857BD76758FD8D7D8571367E6
:102DB0001700D8D79843B7060001558F98C3B717A7
:102DC00002409C4313976700E35B07FEB71702407E
:102DD000D843719BD8C3D84313672700D8C3B7170C
:102DE0000240DC43A18BE5DF8280411106C6993F9A
:102DF000B24041018280411106C6B7170240984394
:102E00001367170098C3D843B706FFE0B106758F64
:102E1000D8C39843B706F7FEFD16758F98C398433D
:102E2000B706FCFFFD16758F98C3D843B70601DFC0
:102E3000FD16758FD8C323A607029843B706F7EA95
:102E4000FD16758F98C33707FF0098C7793FB240CA
:102E50004101828093F8F50093F7050199C3B3E827
:102E6000C800814731A058C910C18507C207C18376
:102E70001D476360F70405473317F700758F75D753
:102E800003230500139827003D4633160601134619
:102E9000F6FF33766600339808013366C8001308DE
:102EA0008002E38205FD13088004E39F05FB18C937
:102EB00065BFA14731A050C958C18507C207C1836A
:102EC0003D476363F70405463316F600758E75D6E5
:102ED000032345003707004061173E970A073D4826
:102EE0003318E8001348F8FF337868003397E80098
:102EF0003367070113088002E38F05FB1308800482
:102F0000E39C05FB10C94DBF82800CC982804CC96F
:102F100082809357650037170240BA9798438546D9
:102F2000B396A600558F98C38280935765003717D4
:102F30000240BA9798438546B396A600558F98C32A
:102F4000828013576500B71702403E9714438547A8
:102F5000B397A70093C7F7FFF58F1CC38280B716FE
:102F60000240DC42370740FF7D17F98F5D8DC8C2F4
:102F700082800111B7070008938707249043D44348
:102F80009847DC4732C836CA3ACC3ECE03A7818187
:102F90003AC493878181DC433EC63AC03EC2B7172C
:102FA0000240DC4389838D8B09476381E706B716AE
:102FB0007A0093860620371602405C429183BD8BCF
:102FC0001810BA9703C707FF33D7E6005C42A18306
:102FD0009D8B0C10AE9783C787FEB355F7005C42FC
:102FE000AD839D8B1010B29783C707FEB357F700D0
:102FF00005466305C50C69C509476305E50C0D4722
:103000006303E50081473E8505618280B717024072
:10301000DC431397F700635C0708B7170240DC57DF
:103020001397F70063500708B7160240D85611836C
:103030003D8B93071700D456A18213F7F600930631
:1030400027004547638EE60437177A0013070720E9
:103050003357F7023307D702B7170240D457BD8A58
:1030600085063357D702B7160240DC42C983BD8BB1
:10307000D442139626006354060093E70701B9462D
:1030800063ECF6028907B386E7023D46E395C7F293
:1030900093171700BA97939617000583BA9621BF26
:1030A000D1465DB737177A001307072075B7371772
:1030B0003D001307079045BF8507F1B7BA87A1B751
:1030C000B68791B7AE8781B7411106C6B7170040E2
:1030D000938707C0630EF508B7170040938707C0B2
:1030E00063E5A702B7070040938707406304F5062E
:1030F000B7170040938707806305F506B7070040C0
:103100006303F504B24041018280B7170040938702
:1031100007406306F506B7370140938707C0630D84
:10312000F500B7170040E31FF5FC13054040F53BE1
:10313000130540403935F9B71305B030FD33130599
:10314000B0300135C1B713050040C5331305004049
:10315000CD3B4DBF13051040C93B13051040D5337F
:1031600055B713052040D13313052040D93B59BF33
:10317000130530405D3B13053040E13361B7130563
:1031800050406533130550406D3BADBF83D70500FC
:103190001CD5B7370140938707C06300F504B70714
:1031A0000040630CF502938707406308F502B717E8
:1031B0000040938707806302F502B71700409387AA
:1031C00007C0630CF5001C41BD9B1CC11C4103D70B
:1031D0004500418BD98F1CC115A01C4193F7F7F80E
:1031E0001CC11C4103D7250013770706D98F1CC1CA
:1031F0001C4103D74500418BD98F1CC19C455CD530
:10320000B71700406301F50293870740630DF5008F
:103210001C4193F7F7CF1CC11C4103D7C50013779E
:103220000730D98F1CC1B7370140938707C06307A8
:10323000F5005C4993E717005CC9828083C7E5000D
:103240001CD9C5BF1C4193E717001CC182801C41DB
:10325000F99B1CC182801C41F59B1CC18280914757
:103260006387F50081E51C41ED9B1CC182801C41F8
:1032700093E747001CC182805C45DD8D4CC5828090
:103280001C49FD8D99C1054582800145828093C509
:10329000F5FF0CC98280F36704308280411106C6B5
:1032A0001375F50FC932B24041018280411106C643
:1032B00022C426C24AC02A842E89B2849532CA8585
:1032C0002285D13AA6852285293CB24022449244E7
:1032D000024941018280B707014083A60740134796
:1032E000F5FFF98E23A0D74083A64740F98E23A28D
:1032F000D74083A68740F98E23A4D74083A6C74032
:10330000F98E23A6D74081CD85476382F502854794
:103310006304F6040DC68947630DF6048280B70680
:10332000014083A70640C98F23A0F640CDB7B7065A
:10333000014083A74640C98F23A2F640C9BFB70703
:10334000014083A68740558D23A4A74083A6C7408C
:10335000758F23A6E7408280B707014083A6874088
:10336000758F23A4E74003A7C740598D23A6A74024
:103370008280B707014003A78740498F23A4E74015
:1033800003A7C740598D23A6A74082803707014075
:10339000832707405D8D2320A7408280B707014027
:1033A00023AAA7408280B77700409843719B98C3B7
:1033B0009843598D88C3F3E7108191E5730050104D
:1033C000F3F710818280F3770430F3E70081730014
:1033D0005010F3F70081F3670430DDB7411106C6E2
:1033E00018411C4B93E717001CCB1C419C4B858B51
:1033F000EDFF0D45EF105043B240410182800111B5
:1034000006CE22CC26CA4AC84EC652C456C25AC09C
:10341000230205008947A300F5002300C50011C65B
:103420008547630CF6080545CDA0B1472301F5009B
:103430009947A301F5008947A302F5003709044025
:103440002E84AA8485472303F500A303F50085672E
:10345000138B07804A9B930A0940130A09449387F8
:1034600007E0B309F9001306C00B81452285EF7010
:103470002059232024012322640123245401232CD6
:103480004407232C340B014783C734006373F704CC
:1034900093175700CA97856693850690BE951316B5
:1034A000270022964CC6938606B0B69793068700EF
:1034B0008A06A296DCC20507C1BFA1472301F50019
:1034C0009147A301F5008947A302F5003709005091
:1034D00085BF814703C7240063F8E702939657002E
:1034E000CA96938606501387C7000A07229754C7C7
:1034F0009396C700CA960567BA961387C7010A074D
:10350000229754C78507F9B70145F2406244D24477
:103510004249B249224A924A024B05618280011116
:1035200006CE22CC2AC42EC632841C42985F98470D
:10353000799B98C70347D1008547630DF70218426E
:103540005C4793E707045CC73285493D8347E10048
:10355000A1EB37072D001C4098DF5145EF10B02D2F
:103560000347C10085476300F7040145F240624408
:10357000056182801C423707100098DF1442DC4648
:103580003707E0FF1307F7FBF98FDCC61442DC4670
:103590003707F0FF7D17F98FDCC632858135C9B753
:1035A00037073D004DBF18401C4793E707021CC773
:1035B00018401C47859B1CC718401C4793E7A70071
:1035C0001CC765B78D06898271060A062A96484689
:1035D0001386F6FF9DC283C7050003C715002207A7
:1035E000D98F03C725004207D98F03C7350062076B
:1035F000D98F1CC19105B286E1BF014582800D06BD
:103600000982685D1307F6FF15C21C412380F5008F
:1036100093D68700A380D50093D607012381D500D8
:10362000E183A381F50091053A86E9BF2E8582806A
:10363000411106C69A051C4193E505028CCB1C413D
:103640009C4B93F70702E5FF0D45EF10F01D014578
:10365000B24041018280411106C61C41414798CBCE
:103660001C419C4BC18BEDFF0D45EF10F01B01453C
:10367000B240410182801C457D57D8C31845B70729
:1036800000C0FD175CCB1845B717008093870780F3
:103690001CCF8347450091E718451C4F93E707016E
:1036A0001CCF14459C4E37370C002907D98F9CCE70
:1036B00018451C4793E717001CC70145828041113C
:1036C00006C622C426C22A841445DC46370700A059
:1036D0007D17F98FDCC618455C47B7060040D58FCB
:1036E0005CC78327050C23A0070054459C427977CB
:1036F0001307F77FF98F9CC25C45984398C35845E0
:103700001C43F19B1CC30347050085476307F70271
:1037100093048400C1452685213F26852D3F5C44C6
:1037200023A807005C4423AA07005C447D5798CF78
:103730005C4423AE0700814779A058451C4393E7BA
:1037400037001CC31C4513070008D8D31845B7071A
:103750004000938707081CD79305000805478D474D
:10376000E3E8E7FA9306F7FFB7C700089387471B1C
:103770008606BE9683D60600B69593161700B697B2
:1037800083D70700C2071444CD8F1306F7030A0638
:10379000B296DCC20507E1B7144337060048D18E64
:1037A00014C33DA8144337060048D18E14C31387B1
:1037B00087000A072297544723A806005847930614
:1037C000F00F14C785070347340063F0E70413972D
:1037D00027002297584B1443E3C006FC2320070020
:1037E000139727002297544B23A80600584B9306A3
:1037F000F00F14C7138787000A072297584714430E
:10380000E3C206FA232007005DB72285AD350145E6
:10381000B240224492444101828058455C4393E780
:1038200027005CC3828058455C43F59B5CC3828063
:1038300058451C4393F7F7801CC358451C43920519
:10384000CD8F1CC38280411102C69C41BD8B3E8836
:1038500003870500634C0706138787000A072A972A
:103860005847138607018546B396C60036C61443EB
:1038700013960601634406041443370634FC13060A
:103880000680F18E14C3631C08045445944613F853
:1038900066001043B7C600089386061BC29683C60F
:1038A0000600D18E14C3144303C615004A06DA0776
:1038B000D18FDD8EB7870010DD8E14C3B246584518
:1038C0005C4FD58F5CCF0145410182801397270063
:1038D0002A97584B8546B396F60036C649BF14431F
:1038E00003D64500D18E14C37DBF9C41BD8B038799
:1038F0000500634807029386070105473317D70081
:10390000A1078A07AA97D0471C42E176FD16F58FDA
:103910001CC25445DC4E1347F7FF7D8FD8CE0145BE
:10392000828005473317F7008A07AA97D04B1C42BD
:10393000E176FD16F58F1CC2E9BF011106CE90415C
:103940003D8A93172600AA97DC4B98433AC69C4BB6
:103950003EC4A247370700E0F98F3EC4DC45BDE313
:10396000A24737070800D98F3EC493172600AA97AD
:10397000DC4B224798CB034745008547630AF7088D
:1039800003C715008547630CF708B2473707008463
:10399000D98F3EC693172600AA97DC4B324798C3AF
:1039A00003C715008547630DF708DC4581CB5445F7
:1039B000DC5A05473316C700D18FDCDA0145F240E7
:1039C000056182801DEA03D745006373F700BA875B
:1039D000DCC5A24737070800D98F3EC4DC45224723
:1039E000D98F3EC403C715008547E310F7F8A247F7
:1039F00037070060D98F3EC48DBF03D74500BA9703
:103A0000FD17B3D7E702CE072247D98F3EC4F9B7D7
:103A100093172600AA97DC4B984DD8CB95B75C45F9
:103A20009C4793F7071099C7B24737070020D98FF3
:103A30003EC6A1BFB24737070010D98F3EC6B1B707
:103A400083D6C5008C452105B53E8DBF9C41BD8BFD
:103A5000138787000A072A970328C7000326080050
:103A600003270801370300E03373670083A8C5000C
:103A70006383080095EF03D7450033676700B706F7
:103A80000800558F2328E800834645000547638FCB
:103A9000E60283C6150005476382E6043707008403
:103AA000598EA1078A07AA97DC4790C301458280F7
:103AB00083D64500B698FD18B3D8D80213973801BD
:103AC00033676700B3861603558F6DBF1387870072
:103AD0000A072A975847944D54CB65BF03C7350052
:103AE00009C737070020598E55BF37070010598E78
:103AF00075B79C41BD8B03870500634D0700A10787
:103B00008A07AA97D8471C43B7062000D58F1CC345
:103B1000014582808A07AA97DC4B3E879443E3D411
:103B200006FE944337060040D18E94C3E9BF9C4102
:103B3000BD8B0387050063460702A1078A07AA9782
:103B4000D4479C423707E0FF7D17F98F9CC283C79B
:103B50001500F91793F7F70F05476378F70001454C
:103B600082808A07AA97D44BE9BF9C42370700108E
:103B7000D98F9CC2EDB75C45884FDC4F7D8D41816C
:103B80001375F5038280A1058A05AA95DC4598473F
:103B90005C45C84B798D82805C45884FDC4F7D8DBC
:103BA0001375F50382805845144B5C5BB3D7B7009F
:103BB0009E0793F7F70FD58F8A052E95584908472A
:103BC0007D8D82805855B7070860E1071CCB0347FD
:103BD000450085476303F7008280130745425C5523
:103BE000D8CB58551C43B7860080D58F1CC3EDB782
:103BF0008347750091CB5C459C47858B91C7032714
:103C0000050C1C43F19B1CC3828018455C4B858BC3
:103C100063950712411106C622C426C2404B1C4FB1
:103C20007D8C79C0AA849317C40063C4070C9317D2
:103C3000D40063C2070C856793870780E18FDDEFAF
:103C40006341040C9377240081C79C440947D8CB77
:103C500093778400B9C383A704439C4F99C32685F7
:103C60008297B707002083C7876A93F7F70F9DC332
:103C7000B70700209387876A03C7070005071377F4
:103C8000F70F2380E70083C7070093F7F70F094773
:103C90006364F7089C442147D8CB93770401C9E7B4
:103CA0009317340163C507089317240163C40708F9
:103CB0009317B40063DC070083A70443DC4F99C368
:103CC000268582979C4437071000D8CB9317A40011
:103CD00063DC070083A704439C5399C3268582971E
:103CE0009C4437072000D8CBB24022449244410183
:103CF0008280A9202DBF26851D2235BF2685CD2E89
:103D000081B783C7740C93F7F70F2383F40C9C449B
:103D100037070080D8CB3DB72685EF00B071B707D5
:103D200000202384076ABDB72685692295BF2685B2
:103D3000A5249DBF2685A926A5BF8280797106D6B8
:103D400022D426D24AD04ECE2A8935352A848144BF
:103D5000A1A0938784008A07CA97DC479C4B3EC684
:103D600013973400058F93172700CA9703D70727A7
:103D7000B246370608007D16F18E158F23AEE72672
:103D8000A1A0A1EC0347C94299476318F7044A85EB
:103D9000153DA1A0058085043DC893771400FDDB87
:103DA00093F9F40FCE854A85F93B2AC4A247858B47
:103DB0008DC7938784008A07CA97D84785471CC751
:103DC00003474900E307F7F8CE854A85EF00506DB9
:103DD000034749008547E306F7FAA247A18BDDDBDD
:103DE000D5F8B707002083C7876A93F7F70FDDD3AD
:103DF0004A85EF003064B70700202384076A938761
:103E000084008A07CA97DC47214798C761B70545F0
:103E1000B250225492540259F2494561828079711C
:103E200006D622D426D24AD04ECE52CC2A89AD33E1
:103E30002A8481441DA893972400CA97DC4B054A25
:103E400023A44701CE854A85EF003073834749009C
:103E5000639A470385E80347C94295476314F7020D
:103E60004A858D3305A00580850405CC9377140021
:103E7000FDDB93F9F40FCE854A8535332AC6B24768
:103E8000858BD5FBB24793F70708F1DFA6854A85F6
:103E9000F52493972400CA97DC4B1307000898C7B2
:103EA000D9B70545B250225492540259F249624A98
:103EB00045618280797106D622D426D24AD04ECE70
:103EC00052CCAA8402C618451C4FBD9B1CCF1C4572
:103ED0009C533EC632491379F9003246118213745D
:103EE000F67FB247BD8313F73700B247C583BD8B5A
:103EF00089466383D70299466389D70498441C4F47
:103F000093E707011CCF0545B25022549254025941
:103F1000F249624A4561828075D0131A3900B307AD
:103F20002A4193992700AA99228683A5492721052A
:103F3000EFF0EFEC83A74927A29723AAF92603A65F
:103F4000C927229623AEC92655BF93163900B386DA
:103F5000264193972600AA9783C7C726BD8BD9FF12
:103F6000A147E31DF4F859FB22869305454221053C
:103F7000EFF0EFE893173900B38627411397260037
:103F800026970326C7272296232EC726B707002089
:103F900005472384E76A9DB7411106C622C426C29D
:103FA0004AC02A8458455C43F99B5CC3814521057E
:103FB000EFF00FE80147834734006371F70293176E
:103FC0002700A297DC4B9306F00F94C79307870056
:103FD0008A07A297DC4794C70507F1BF5C447D5769
:103FE00098CF5844C16785075CCF5C442547D8CB40
:103FF0005C44854484CB58441C4393F7F7801CC32E
:10400000A302040C22857D3E1C440567D8CB2326E1
:10401000042623280426232A0426232C0426232EC0
:10402000042623200428232204281309000423182B
:1040300024279305C4262285EFF0FF802324040C57
:104040002326040C2328040C232A040C232C040C00
:10405000232E040C2320040E930700F82304F40CF1
:104060002316240D9305840C2285EFF0CFFD230346
:10407000940C0545B2402244924402494101828099
:1040800054459C46858313F73700DC4293F7F7EFDE
:10409000DCC25445DC4293E70710DCC210455C46A5
:1040A000F1769386F63FF58F5CC6B7C70008938715
:1040B000C71BBA9703C707008D476301F7028947FB
:1040C000A300F5001445DC46056713070740D98FA8
:1040D000DCC61C450967D8CB05458280A300F500E6
:1040E0001445DC46096713070740D98FDCC6D5B7EE
:1040F000011106CE22CC2A8483477500A307F10064
:104100005C459C47858B2307F1008347650C93F73B
:10411000F70F0D476387E7048147A306F100834744
:10412000640C93F7F70FA303F40C91472303F40CEB
:104130008347F10093F7F70F99CB8347E10093F79B
:10414000F70F91C78347D10093F7F70F89EF184412
:104150008567938707805CCB0545F2406244056123
:10416000828085475DBF0327040C1C4393E737001B
:104170001CC381450545EFF00FA3D1BF011106CE49
:1041800022CC26CA4AC84EC652C4AA892E89139781
:1041900035000D8F93172700AA9703A7470D83A615
:1041A000870D158F03DAC70C6363EA003A8A0D0A9C
:1041B000135A2A00A9A0138A3400135A2A0093170D
:1041C0003900B3872741139427004E949396040136
:1041D000C1821376F90F8325040D13858900EFF052
:1041E0006FBE8327040DA6972328F40C8327840D24
:1041F000BE94232C940C8327440D6386F4049317F8
:104200002900CE97DC4B9C4FC207C1836378FA0428
:10421000131739003307274193172700CE9703A7B9
:10422000870D83A7470D637BF702998F931639009B
:10423000B3862641139726004E978354C70CE3ECB0
:10424000F4F6BE848DBF83A6C900D85A8547B397BC
:10425000270193C7F7FFF98FDCDA55B70545F24020
:104260006244D2444249B249224A056182804111E6
:1042700006C603C7250003C8450083C75500A2072B
:1042800033E8070193178701E18763C30706131615
:104290003700B306E64093972600BE86938707262D
:1042A000AA97B107AA9603C6C6261376F6072386F1
:1042B000C6263D8B83C60700C19A558F2380E70031
:1042C0001377F80F2392E70003C735000D8B931681
:1042D0002700370700081307072536971843A380E0
:1042E000E700BE85EFF02FD60145B2404101828044
:1042F0009378F70713963800B30716419396270073
:104300009386060CAA969387860033061641931669
:104310002600AA9603C6860C136606F82384C60CEC
:1043200049BF411106C693978501E18763C2070221
:1043300093973500B385B74093972500938507265B
:10434000AA95B105EFF06FDA0145B24041018280D4
:1043500093F5F507939735008D8F939527009385F7
:10436000050CAA95A105F9BF411106C613F8F5077A
:1043700013173800B3050741939725009387072645
:10438000AA979385C7003307074193172700AA9779
:1043900023AAC72623ACD72623AE0726034745000A
:1043A00085476308F700EFF06FEA0145B24041012D
:1043B0008280931738003388074193172800AA9703
:1043C00023A2C728CDB7411106C613F8F507131766
:1043D0003800B3050741939725009387070CAA97E8
:1043E000938587003307074193172700AA9723A8CF
:1043F000C70C23AAD70C23AC070C034745008547FD
:104400006308F700EFF06FD30145B24041018280AD
:10441000931738003388074193172800AA9723A0E1
:10442000C70ECDB7411106C693978501E18763C5D5
:10443000070293973500B385B7409397250093857E
:104440000726AA95B10585472381F500EFF06FEAAD
:104450000145B2404101828093F5F50793973500FD
:104460008D8F939527009385050CAA95A105E1BF33
:10447000411106C693978501E18763C407029397AC
:104480003500B385B7409397250093850726AA95F5
:10449000B10523810500EFF08FE90145B2404101EC
:1044A000828093F5F507939735008D8F93952700BC
:1044B0009385050CAA95A105E9BF411106C6EFF049
:1044C0002FB7B2404101828093973500B385B74042
:1044D000939725003E950355C5278280411106C656
:1044E000EFF06FB40D45EF001035B240410182800E
:1044F000411106C6EFF06FB20D45EF00D033B24068
:1045000041018280411106C622C426C22A84232882
:10451000C542930485002E86A685EFE05FEE2686D1
:1045200008404C40EFE0BFFF2285D9372285EFF0ED
:104530000F992285653785472303F40CB240224446
:10454000924441018280054582808327454183C78B
:1045500007002310F600032545418280832785410B
:1045600083C727002310F600032585418280832717
:10457000C54183C727002310F6000325C54182806B
:10458000832705428A05AE97884383470500231099
:10459000F600828003C7450083C75500A207D98F64
:1045A00013F6F70F03C705000D8B85466305D70883
:1045B00093168701E18691C689466307D70A0545A8
:1045C00082808347650C93F7F70F0947638BE700F9
:1045D0008347650C93F7F70F0D476384E7000545A4
:1045E00082808347054195CFB70700200547238682
:1045F000E76A834725419DCBB70700209387C76AA9
:1046000003C70700136727002380E700B7070020D0
:104610009387C76A2328F50C8947232EF50C01459B
:104620008280B70700202386076AE1B7B70700201A
:104630002386076AE1BF8347650C93F7F70F0D47A1
:104640006384E70005458280854763F4C70005451C
:104650008280B70700209387C76A2328F50C894713
:10466000232EF50C014582800347650C1377F70F65
:104670008D466304D70005458280E207E18763CA5F
:104680000702931736003386C74093172600AA9770
:1046900003C7E726B70700202386E76AB70700208D
:1046A0009387C76A2328F50C8947232EF50C01450B
:1046B00082801376F607931736003386C740931728
:1046C0002600AA9703C7A70CB70700202386E76A2E
:1046D000F1B7411106C622C426C2AA842E8483C71C
:1046E00005008D8B85C305476386E70C03A7C40DC2
:1046F00065CB8346640083477400A207D58FE1E34E
:104700000545C5A083C7250083C53500A205DD8DFD
:1047100093D7850093F5F50F0947638EE704637E11
:10472000F7000D476387E7063D47E391E7FC130673
:10473000C50D353D23A8A40C55BF0547E398E7FAFE
:10474000FD178A073707000813074729BA979C43C4
:104750001306C50D829723A8A40C03476400834762
:104760007400A207D98F13070004E391E7F8A1476B
:1047700023AEF40CA5BFFD178A07370700081307FF
:104780004729BA979C431306C50D829723A8A40C0A
:10479000B1BF1547E36CB7F4FD178A073707000868
:1047A00013074729BA979C431306C50D829723A880
:1047B000A40C2DBF83270543DC4782971DA0637D92
:1047C000F70083D7C40C636BF7003377F70219E760
:1047D0008547A386F44219A023AEF40C014511A02D
:1047E0000545B240224492444101828001458280C5
:1047F0008347650C93F7F70F09476387E7000D4779
:104800006382E702054582808347450C99C30545CD
:1048100082809307450C2328F50C8547232EF50C41
:10482000014582808347450C99E3054582809307C3
:10483000450C2328F50C8547232EF50C0145828075
:1048400083C52500B7070020A384B76A854763F4B2
:10485000B70005458280411106C622C42A848347D9
:10486000650C93F7F70F0947638AE7000D476387E5
:10487000E7020545B24022444101828091CD832761
:104880000543DC438297B707002083C7976A23025A
:10489000F40C8D472303F40C0145E9BF85E1832720
:1048A00005439C478297B707002083C7976A230276
:1048B000F40C89472303F40C01456DBF8347450C75
:1048C000E38CF5FE832705439C478297B7070020BA
:1048D00083C5976A2302B40C83270443DC432285F3
:1048E0008297D9BF8347650C93F7F70F0D47638411
:1048F000E7000545828003C74500854763F4E7006C
:10490000054582808327054385072328F50C8547C5
:10491000232EF50C014582808347650C93F7F70F32
:104920000D476384E7000545828003C7450085473E
:1049300063F4E7000545828003C72500832705430C
:10494000A380E700014582800145828003C74500BE
:1049500083C75500A207D98FB9EB03C7650083C78A
:104960007500A207D98FB1E783C5250093F5F50738
:10497000A302B50C8347650C93F7F70F0D476394BB
:10498000E70005458280411106C622C42A843536D7
:104990008347540C89CB89472303F40C0145B2406B
:1049A00022444101828085472303F40CC5BF05459D
:1049B00082800545828083C705008D8B91C709479A
:1049C0006383E704054582808347650C93F7F70FFF
:1049D0000947638BE7008347650C93F7F70F0D4793
:1049E0006384E7000545828003C7250083C735003F
:1049F000A207D98F05476384E70001458280854778
:104A00002309F540DDBF83C645008347650C93F756
:104A1000F70F0D476384E7000545828003C7250033
:104A200083C73500A207D98F91E789C6930700088D
:104A30006394F60001458280411106C6B685DD32D9
:104A40000145B2404101828083C705008D8B91C72B
:104A500009476383E704054582808347650C93F724
:104A6000F70F0947638BE7008347650C93F7F70F50
:104A70000D476384E7000545828003C7250083C78F
:104A80003500A207D98F05476384E700054582807A
:104A9000230905400145828083C645008347650C94
:104AA00093F7F70F0D476384E7000545828003C73E
:104AB000250083C73500A207D98F91E789C69307E0
:104AC00000086394F60001458280411106C622C4A5
:104AD00026C22E84AA84B685EFF09F9983A704434B
:104AE000DC47A285268582970145B2402244924444
:104AF00041018280411106C683C715001397270024
:104B0000B707000893870726BA979C438297B2405D
:104B1000410182808347650C93F7F70F0D4763844B
:104B2000E7000545828003C74500854763F4E70039
:104B300005458280411106C683270543DC478297DD
:104B4000B2404101828001458280411106C622C4E3
:104B50002A8493050008EFF0FF8C81452285EFF051
:104B60007F8C2285EFF00F86B24022444101828083
:104B7000411106C622C42A848356C50D0326050D9D
:104B80008145EFF05F840327C40D8357C40C63FA9B
:104B9000E70085472306F4420145B2402244410123
:104BA000828089472306F442C5BF411106C622C44C
:104BB0002A8483560528032645278145EFF0CFFA3E
:104BC000032704288357042763FAE7008D47230649
:104BD000F4420145B24022444101828091472306BC
:104BE000F442C5BF411106C622C42A849547230654
:104BF000F542814601468145EFF0EFFC2285EFE06A
:104C00007FFC0145B240224441018280411106C629
:104C100022C42A8499472306F542814601468145EC
:104C2000EFF08FF42285EFE0FFF90145B240224416
:104C300041018280011106CE22CC2A84832745427D
:104C40003EC4032785423AC693F7070613070002BE
:104C5000638CE70213070004638BE70289CB2C0007
:104C60002285E5350145F2406244056182802C00D1
:104C7000513575F58357E10091CF8307810063CEED
:104C8000070022851D37F9BF2C006935DDB72C00E0
:104C90005D3DC5B72285B937F1B72285D13DD9B77A
:104CA000797106D622D40018232EA4FCAE87A30D5A
:104CB000F4FC8347B4FDD1E38327C4FD9387C72663
:104CC0002326F4FE8327C4FD83C7C7420D476386AE
:104CD000E70011476383E70259A88327C4FEDC4B32
:104CE0000327C4FE035747003387E7408327C4FEEA
:104CF000D8CB0325C4FD553D9DA88327C4FD83C79C
:104D0000670C13F7F70F8D476311F7028327C4FD74
:104D100083A70743DC4B91CB8327C4FD83A70743BD
:104D2000DC4B81450325C4FD82978327C4FE23AA5B
:104D300007000325C4FD7D351DA88327C4FD83A777
:104D40000743DC4B8DC78327C4FD83C7670C13F76C
:104D5000F70F8D47631DF7008327C4FD83A7074323
:104D6000D84B8347B4FDBE850325C4FD0297814718
:104D70003E85B250225445618280797106D622D494
:104D80000018232EA4FCAE87A30DF4FC8347B4FDCA
:104D9000DDE38327C4FD9387870C2326F4FE832756
:104DA000C4FD83C7C74205476386E700094763839D
:104DB000E70265A88327C4FEDC4B0327C4FE035724
:104DC00047003387E7408327C4FED8CB0325C4FDC3
:104DD000453361A88327C4FD83C7D74289CF814665
:104DE000014681450325C4FDEFF0EFDD8327C4FDB7
:104DF000A38607429DA88327C4FD83C7670C13F7CA
:104E0000F70F8D476311F7028327C4FD83A707437C
:104E10009C4B91CB8327C4FD83A707439C4B8145C3
:104E20000325C4FD82978327C4FE23AA0700032518
:104E3000C4FDE93B1DA88327C4FD83C7670C13F796
:104E4000F70F8D476313F7028327C4FD83A707433A
:104E50009C4B81CF8327C4FD83A70743984B83478F
:104E6000B4FDBE850325C4FD029781473E85B2503F
:104E7000225445618280011106CE22CC2A8413057A
:104E80001070EFE00F893705004013050540EFE093
:104E9000AFA389476305F40685476305F406B72782
:104EA000002083A7C7922310F100231101002312D1
:104EB000010023160100230701008A853704004002
:104EC00013050440EFE08FAC13050440EFE0AFB8EA
:104ED000854513050440EFE02FBA854513050440CE
:104EE000EFE0EFBA814513050440EFE04FB713053B
:104EF0000440EFE02FB5F240624405618280AD4787
:104F00003EC471BF8D679387F7ED3EC449BF411121
:104F100006C6B707002023A8A76A2E85A93FB707B2
:104F2000002083A7076BE5FF370500401305054008
:104F3000EFE0EFB1B24041018280411106C6014568
:104F4000EFE02F83B777DC02938707C0630AF5028F
:104F5000B7A74A0493870720630CF504B7E7B805A1
:104F6000938707806319F502B70700203707C00051
:104F700023AAE76AB72700201D4723A6E79221A8A6
:104F8000B70700203707400023AAE76AB7270020A9
:104F90000D4723A6E792B707002003A5476BEFD084
:104FA0001FFC1305C050EFD0DFF6B24041018280F4
:104FB000B707002023AA076AB7270020154723A6B2
:104FC000E792D1BF411106C601468545130560052C
:104FD000EFE0CFAD1305C071EFD0BFF3370504008C
:104FE000EFE0CFBB0146814537050400EFE0AFAEEF
:104FF00037050400EFE08FB901468D451305D00356
:10500000EFE0CFAAB24041018280411106C61305EC
:105010001070EFD01FF00146894513050003EFE043
:10502000EFA8B24041018280411106C68945C535CD
:10503000B24041018280411106C68545C93DB2405A
:1050400041018280411106C68545370500401305A0
:105050000540EFE0EFA201E5B240410182808545C5
:105060003705004013050540EFE06FA2B7070020A9
:1050700083A7076B89CBB70700209387076B9843FB
:105080007D1798C3D1BF3705004013050540EFE0F9
:105090000F9CD9B7411106C63705002013058506B8
:1050A000EFE0BFB6B240410182808280411106C666
:1050B000B70700209387870683C7770081EB370502
:1050C0000400EFE0AFADB24041018280EFD0BFD22B
:1050D000B707002003A5476BEFD07FE81305C0504A
:1050E000EFD03FE33705002013058506EFE05FB002
:1050F000F9B7411106C6B937B2404101828041116A
:1051000006C622C426C2AA84370400201304040061
:105110009305C403EFF0AF95930554032685EFF094
:105120000F95930554022685EFF06F940145B24028
:105130002244924441018280411106C622C42A843D
:1051400093051008EFF0EF9D8D452285EFF06F9DE0
:10515000930520082285EFF0CF9C0145B240224400
:1051600041018280411106C681C98D476389F500DE
:105170000945B2404101828001220945DDBF054752
:105180002388E1808D45EFF02FB4B707002023ACD2
:10519000A76A0145F9BF85476384F5000945828008
:1051A00093F6F507939736003386D74013172600FA
:1051B0002A970326470D958F139727002A97835721
:1051C000C70CB377F60291E311E60547A388E180A7
:1051D00001458280411106C681460146EFF0AF9E2F
:1051E0000145B2404101828083C7150013070002C8
:1051F0006388E700130710026385E7020145828098
:1052000023A2F180B727002093870797232AF5264A
:1052100003C7650083C77500A207D98F2320F5282F
:10522000F1BF138781801443B72700202388D796C6
:1052300013D6860093870797A380C70013D606016D
:105240002381C700E182A381D700834647002382E0
:10525000D70083465700A382D70003476700238304
:10526000E7002328F50C03C7650083C77500A20774
:10527000D98F232EF50C59B703A741809307F00F60
:105280006307F704B727002003C70797938707979B
:1052900083C61700A206558F83C62700C206558F06
:1052A00083C63700E206558F9386818098C203C774
:1052B00047002382E60003C75700A382E60083C7A6
:1052C00067002383F6001307F00F23A2E180014556
:1052D0008280411106C6B70700209387476C239050
:1052E000070023910700EFD01FFB0945EFD01FFBFC
:1052F000A931213BC13937060020130646048545F4
:105300003705002013058506EFF0CF9FB24041011D
:105310008280411106C6B707002083D7476C130768
:105320009003638BE7066372F7061307F00363824B
:10533000E70413071004639EE706B707002083A560
:10534000876B13858184EF30C0622DC9238801806B
:1053500093060004138681848D45370500201305CC
:105360008506EFF06F80B70700201307F003239244
:10537000E76C03C7018185476315F704B707002071
:10538000130710042392E76C4DBF85E7B707002091
:10539000130790032392E76CB707002093878706D3
:1053A00083C7670C93F7F70F0D47E381E7FA0145D1
:1053B00031A0B70700202392076C0D45B240410190
:1053C00082800145E5BF411106C622C4B70700200F
:1053D0009387476C83D727001307C004638FE702C6
:1053E0006374F7021307F004638CE70413074005A6
:1053F000639BE70803C7118185476303F7080145ED
:10540000B240224441018280BDEFB707002093875C
:10541000476C1307C0042391E700B7070020938768
:10542000870683C7670C93F7F70F0D476395E70669
:10543000B70700209387476C1307F0042391E70018
:10544000370400201304446C13058400EF304063DC
:1054500048C021C5A3880180370400201304446C90
:10546000835684002A86930510083705002013050B
:105470008506EFE05FF5930740052311F4009DBF1B
:10548000EF30A06175B7B70700209387476C239171
:1054900007000D45B5B70145A5B7014595B74111C1
:1054A00006C6F32700B8732500B0F32500B8E39AC9
:1054B000B7FE130600068146EF50A00FB24041012F
:1054C0008280011106CEE1659385056A2800EF40D0
:1054D000F07721A02800EF40F0780545592A2800F0
:1054E000EF40F0786DDD2800EF40D0770145512284
:1054F0002800EF40D0776DDDF1BF411106C622C410
:10550000938781882390070023810700A3810700E8
:1055100013052060EFD0FF9F13054060EFD07F9F01
:1055200091460946C1453714014013050480EFD068
:105530007F92914513050480EFD03F9D894609462F
:10554000C14513050480EFD0FF9089451305048001
:10555000EFD0BF9B89660946C14537150140EFD0A2
:105560007F8F896537150140EFD03F9AB2402244C2
:1055700041018280411106C683D7818813079004B8
:105580006385E7081307D004638CE70A99C723945F
:1055900001880D45B240410182809387818883C78D
:1055A000270085CB9387818883C7370091CB93876A
:1055B00081883797980013070768D8C398C735A024
:1055C0009387818837F7FA0213070708D8C398C76B
:1055D00029A8938781883797980013070768D8C34D
:1055E00037E7F5051307071098C7894537150140B8
:1055F00013050580EFD0BF91732700B09387818892
:10560000D8C7130790042390E700732700B093874F
:105610008188D447158FDC436374F70001459DBF33
:1056200089453715014013050580EFD01F8E73277C
:1056300000B093878188D8C71307D0042390E70070
:10564000732700B093878188D447158F9C47E370F8
:10565000F7F4014581B73335A00093878188238112
:10566000A70082803335A00093878188A381A7009B
:105670008280411106C609E9896537150140EFD0DE
:10568000DF88B24041018280896537150140EFD043
:105690001F88C5BF411106C622C413052060EFD084
:1056A0005F8713053060EFD0DF8613050060EFD011
:1056B0005F86B7060140DC42370700F97D17F98F96
:1056C00037070004D98FDCC291660546C1453714FF
:1056D000014013050480EFD0EFF789660546C14508
:1056E00013050480EFD00FF7A1660546C1451305E9
:1056F0000480EFD02FF6A1460146930580041305E0
:1057000004C0EFD02FF5B240224441018280411104
:1057100006C622C49166014681453714014013052F
:105720000480EFD02FF3896601468145130504807C
:10573000EFD04FF2A1660146814513050480EFD0FA
:105740006FF1A14601468145130504C0EFD08FF0EB
:10575000930600200146814513050480EFD08FEFAA
:10576000B240224441018280411106C622C419CDB3
:105770009306002001468145371501401305058039
:10578000EFD04FEDB24022444101828093050020CA
:105790003714014013050480EFD06FF79306002003
:1057A0000546D14513050480EFD0CFEAE1BF411192
:1057B00006C6CD35B7170140096723A8E780B24078
:1057C000216723A8E780116723AAE780410182802F
:1057D0003DBFB7170140096823AA0781216823A8A4
:1057E0000781732800B0F32700B0E30EF8FEB71767
:1057F0000140116823A8078183A787C0F32800B060
:105800007548F32700B0B3871741E37CF8FEB7175C
:105810000140116823AA0781096823AA078121682A
:1058200023A80781732800B0F32700B0E30EF8FE29
:10583000B7170140116823A8078183A787C0F32801
:1058400000B07548F32700B0B3871741E37CF8FE3A
:10585000B7170140116823AA07818148A1C63718EC
:105860000140930E48818962A16F116E754F23A08C
:105870005E002328F881732300B0F32700B0E30E05
:10588000F3FE2328C881832788C0732300B0F32741
:1058900000B0B3876740E37CFFFE23A0CE018508FC
:1058A000E397D8FC130FF6FF01486305061E41116C
:1058B00022C626C4371301408962916E754EA163DA
:1058C000854F935658008A06B387D50083A80700F2
:1058D0009377F801B3D8F80093F8180063140F0118
:1058E000630B0716232A53806388081223287380CA
:1058F000732400B0F32800B0E30E14FF2328D381F3
:10590000832883C093D8380093F81800F32400B09C
:10591000732400B0058CE37D8EFE232AD381AA96E2
:10592000B397FF0080426384080EC18F9CC20508B4
:10593000E31906F99308F7FF014621C7B71701409D
:10594000096E21631165F545638BC80C23AAC781D5
:1059500023A86780732800B0F32600B0E30ED8FEBA
:1059600023A8A78083A687C0732800B0F32600B0C1
:10597000B3860641E3FCD5FE23AAA7800506E315FE
:10598000E6FCB7170140096723A8E780216723A831
:10599000E780732700B0F32700B0E30EF7FEB717D8
:1059A0000140116723A8E78083A787C0F32600B0D2
:1059B0007547F32700B0958FE37DF7FEB7170140D9
:1059C000116723AAE780096723AAE780216723A834
:1059D000E780732700B0F32700B0E30EF7FEB71798
:1059E0000140116723A8E78083A787C0F32600B092
:1059F0007547F32700B0958FE37DF7FEB717014099
:105A0000116723AAE7803244A2444101828093C7F0
:105A1000F7FFE18F9CC221BF232A7380D1BD23A849
:105A2000C78123A86780732800B0F32600B0E30E77
:105A3000D8FE23A8A78083A687C0732800B0F326CA
:105A400000B0B3860641E3FCD5FE23AAA780050675
:105A5000E31CE6EE3DB723285380638A080223281F
:105A60007380732400B0F32800B0E30E14FF2328E2
:105A7000D381832883C093D8380093F81800F32487
:105A800000B0732400B0058CE37D8EFE79B5232A27
:105A90007380C1BF9308F7FF014621C7B7170140C4
:105AA000096E21631165F5456380C80C23AAC7817F
:105AB00023A86780732800B0F32600B0E30ED8FE59
:105AC00023A8A78083A687C0732800B0F32600B060
:105AD000B3860641E3FCD5FE23AAA7800506E3159D
:105AE000E6FCB7170140096723A8E780216723A8D0
:105AF000E780732700B0F32700B0E30EF7FEB71777
:105B00000140116723A8E78083A787C0F32600B070
:105B10007547F32700B0958FE37DF7FEB717014077
:105B2000116723AAE780096723AAE780216723A8D2
:105B3000E780732700B0F32700B0E30EF7FEB71736
:105B40000140116723A8E78083A787C0F32600B030
:105B50007547F32700B0958FE37DF7FEB717014037
:105B6000116723AAE780828023A8C78123A86780C2
:105B7000732800B0F32600B0E30ED8FE23A8A78058
:105B800083A687C0732800B0F32600B0B386064111
:105B9000E3FCD5FE91B7B7170140096723A8E7805A
:105BA000216723A8E780F32700B0732700B0E38EB6
:105BB000E7FEB7170140116723A8E78083A787C0D6
:105BC000F32600B07547F32700B0958FE37DF7FE0D
:105BD000B7170140116723AAE780054781466FF098
:105BE0005FBFB7170140096723A8E780216723A893
:105BF000E780F32700B0732700B0E38EE7FEB71706
:105C00000140116723A8E78083A787C0F32600B06F
:105C10007547F32700B0958FE37DF7FEB717014076
:105C2000116723AAE780096723A8E780216723A8D3
:105C3000E780F32700B0732700B0E38EE7FEB717C5
:105C40000140116723A8E78083A787C0F32600B02F
:105C50007547F32700B0958FE37DF7FEB717014036
:105C6000116723AAE780154781466FF09FB6371763
:105C700001401946930607810963A16811657548BB
:105C800023A0660023A01601F32500B0F32700B07F
:105C9000E38EF5FE88C2832787C0F32500B0F32783
:105CA00000B08D8FE37DF8FE93074781232AA780FC
:105CB0007D1679F6896694C3A1672328F780732738
:105CC00000B0F32700B0E30EF7FEB71701401167ED
:105CD00023A8E78083A787C0F32600B07547F32782
:105CE00000B0958FE37DF7FEB7170140116723AA37
:105CF000E780828021C5371701408146130847811C
:105D0000096E21639165F5482320C8012328678027
:105D1000732600B0F32700B0E30EF6FE2328B78009
:105D2000832787C0732600B0F32700B0918FE3FD6F
:105D3000F8FE2320B8008506E318D5FC82803705DD
:105D400000081305453282800965130585D18280DC
:105D5000937735000D476383E7021357B500718BC6
:105D6000D98F1387C7FFE94663E9E6080A07B72614
:105D70000008938606043697184302879377F50741
:105D80001D476381E7046378F702130730026386D7
:105D9000E700130770026393E7029357F500FD8B4A
:105DA0009CC1B70700FEE98F36053707F001798DF2
:105DB0005D8D518529A80D476386E70023A0050066
:105DC000014531A09357F500FD8B9CC1518508C258
:105DD0008280135775001D8B210798C1F117694701
:105DE0006362F70A8A07372700081307C70ABA97BA
:105DF0009C438287094798C1D5B723A00500F9BF06
:105E00009357750093F7870306051375050C5D8D91
:105E10007DBF9357750093F7870313574500118B88
:105E2000D98F0605137505045D8D55B79357750019
:105E300093F7070213572500618BD98F120513754D
:105E4000051C5D8D69B79357750093F707021357CB
:105E50002500718BD98F12051375050C5D8D85BFDB
:105E60009357750093F7870305811375051C5D8DA6
:105E7000B9BF9357750093F7C70305811375050CD8
:105E80005D8DB1B70145A1B7411106C622C42A8470
:105E900083D781891307900B6386E7146363F70246
:105EA0001307900A6382E70E1307F00A6383E71073
:105EB0006388070C239C01880D45B24022444101B0
:105EC00082801307F00C638AE7041307500D638B7D
:105ED000E7061307F00BE39FE7FC938581891386A0
:105EE000C5109385C5044145EF10F06E854763F3F7
:105EF000A7189387818983A7C710639C071293878C
:105F00008189FC47858B639C0712938781890547AC
:105F1000F8C71307F00C2390E70093878189138655
:105F2000C710EC474145EF10D07C854763F6A714B6
:105F30009387818983A7C710639907101307500DB2
:105F4000239CE188938581891386C5109385C504B8
:105F50004145EF105068854763F2A7129387818906
:105F600083A7C7106399070E93878189F8478547F0
:105F70006309F70E8D471CC0239C0188094535BF76
:105F80001307900A239CE188138581891305C511A5
:105F9000EF10B03B854763F9A70C9387818983A7EE
:105FA000C711FD1775576364F7061307F00A239CA2
:105FB000E1881385818913050512EF109048854704
:105FC00063F6A70A9387818983A70712BD8B0547CC
:105FD0006395E7049387818923A607041307900B31
:105FE0002390E700938781891386C710EC474145CA
:105FF000EF103070854763FDA7069387818983A7DB
:10600000C71095E31307F00B239CE188F9B585478A
:106010001CC0239C018809454DB589471CC0239CA1
:106020000188094559BD8D471CC0239C018809453D
:1060300069B58D471CC0239C01880945BDBD8D47AE
:106040001CC0239C018809458DBD8D471CC0239C25
:10605000018809459DB58D471CC0239C01880945D1
:10606000A9BD23200400B9B5014581BD0145B1B5E5
:106070000145A1B5014591B5014581B5014535BD44
:10608000411106C6EF105054B2404101828006878C
:106090009387818923AEE71223ACA7128280411136
:1060A00006C622C426C22A849387818983D7270003
:1060B00013076038638BE7066373F7041307C03870
:1060C000638EE70C1307F0386391E70293858189AB
:1060D0001386C510F1051145EF10F04F854763F3A6
:1060E000A70E93878189DC4F1CC0938781892391F8
:1060F00007000D45B2402244924441018280B9CF4D
:1061000013074038E393E7FE938781891386C7100E
:10611000AC575D45EF10F05D854763FFA708938797
:106120008189130760382391E7009385818913865D
:10613000C510938545065945EF10F049854763FF23
:10614000A70693878189FC5393F7077085E79387A8
:1061500081891307F0382391E7008DBF93878189E8
:1061600037072200B8D72394B70613074038239186
:10617000E70059BF93848189FC50A1839D8B8A07D6
:10618000370700201307C749BA9788430937930791
:106190000070FCD09307C0382391F4009387818965
:1061A0001386C710EC535945EF10B054854763F977
:1061B000A700FD571CC015BF01452DBF01451DBFE0
:1061C00001450DBF01453DB7411106C622C4938765
:1061D000818983D727001307303A638CE7062E8422
:1061E000637EF7021307503A6386E7081307B03A55
:1061F000639DE700938781891386C710EC53594547
:10620000EF10304F854763FBA70C9387818923915B
:1062100007000D45B240224441018280DDC31307CF
:10622000B039E394E7FE138681891306C610AA8568
:106230001145EF10104C854763FCA70893878189AF
:1062400037072300B8D7239487061307303A2391E2
:10625000E700938781891386C710AC575D45EF101F
:106260005049854763F8A706938781891307503AF9
:106270002391E700938581891386C5109385450690
:106280005945EF105035854763F8A70493878189F6
:10629000FC5393F70770B5DB138481897C50A1838D
:1062A0009D8B8A07370700201307C749BA97884391
:1062B000F93B930700707CD09307B03A2311F400A8
:1062C00015BF938781891307B0392391E700A1BFD8
:1062D000014589B701453DBF01452DBF01451DBFA2
:1062E000411106C622C483D781891307900F6380AA
:1062F000E70C2A846372F7061307F00F638FE70237
:1063000013070010639FE70C9305107A01456D3D5C
:10631000854763F5A70E9387818903A707110507B2
:1063200023A8E7109387818903A707118D4763EAA4
:10633000E70A1307F00F239CE1889305007A9387FF
:10634000818903A507114935854763F7A70A130714
:106350000010239CE1884DBFB5CB1307D00E63928C
:10636000E7089305007B1385818913058511EFF0FC
:106370001FD3854763FEA7069387818903A78711EB
:10638000B70700F0F98F370700406396E7041387DB
:10639000818983278711A166D58F8966D58F856608
:1063A000D58F232CF7109307900F2310F700930538
:1063B000007B9387818903A587113935854763FB66
:1063C000A7029387818923A80710A9BF1307D00EBE
:1063D000239CE18879B789471CC0239C0188094523
:1063E00021A0239C01880D45B240224441018280B6
:1063F0000145DDBF0145CDBF0145FDB70145EDB705
:10640000411106C683D781891307E0106382E70430
:10641000637BF70213072011638AE7061307A011B5
:10642000639DE700938781891386C710EC47414538
:10643000EF10302C854763F3A708239C01880D4596
:10644000B24041018280F5FB1307E010239CE188F4
:106450009305007B1385818913058511EFF03FC4F7
:10646000854763F9A7041387818983278711E1761C
:10647000FD16F58FF976FD16F58FFD76FD16F58F75
:10648000232CF710930720112310F7009305007BAE
:106490009387818903A58711EFF01FD3854763FD9B
:1064A000A7009387818923A607041307A0112390CF
:1064B000E7008DBF014569B7014559B7014549B7A7
:1064C000011106CE22CC26CA4AC84EC6AA892E89F8
:1064D000B28436849387818983D727001307E03DF0
:1064E000638CE70A637AF7021307503E638EE71066
:1064F0001307B03E6382E7161307203E6385E70C5F
:1065000093878189239107000D45F2406244D2446C
:106510004249B24905618280638D07141307003C2C
:10652000E390E7FE938581891386451393850513D0
:106530001545EF10A079854763F4A71A93878189E1
:1065400083A7471189CB05476302E4160947630D0A
:10655000E416630404149387818983A74711638F2A
:1065600097089387818923A407060947A385E7062F
:106570001377740093164701B857370690FF7D16BE
:10658000718F558FB8D723A8E712094723AAE712BE
:106590001307E03D2391E700938581891386451316
:1065A000938505135D45EF106072854763FCA71264
:1065B0009387818923A80712054723AAE7121307A7
:1065C000203E2391E70093858189138645139385A7
:1065D00005131145EF10806F854763F7A710938768
:1065E000818903A74711050723AAE71093878189AB
:1065F00083A747111387140063E2E7089387818913
:106600001307503E2391E700938581891386C510B7
:10661000938545065945EF10007C854763F8A70C24
:1066200093878189FC5393F70770E38B07EC1384FE
:1066300081897C50A1839D8B8A073707002013072F
:10664000C749BA978843EFF09FA4930700707CD0A6
:106650009307B03E2311F400938781891386C710F6
:10666000EC535945EF10F0088547E3EBA7E80145E7
:1066700069BD9387818923AA07108DBFB3978700CF
:10668000CA97138781892328F7128947232AF7128B
:106690009307003C2311F70071B513878189032705
:1066A0000713FD17CE972380E70075B513878189FF
:1066B00083260713370700801347F7FFBA9786072B
:1066C000CE972390D70041BD370700407D17BA977A
:1066D0008A07CE97138781890327071398C3A5BD1F
:1066E000014525B5014515B5014505B5014531BD46
:1066F000011106CE22CC26CA4AC84EC62A89AE89C6
:10670000B28436849387818983D727001307E043B7
:106710006381E708637AF7021307A0446383E710F5
:10672000130700456387E71413077044638CE70A77
:1067300093878189239107000D45F2406244D2443A
:106740004249B2490561828063820714130790426F
:10675000E390E7FE9385818913864513938505139E
:106760001545EF10A056854763F2A718630DF41482
:1067700089476304F416630F041293878189D84F05
:1067800023A8E712094723AAE7121307E04323913E
:10679000E700938581891386451393850513114579
:1067A000EF10C052854763F5A7149387818923A40E
:1067B00007060947A385E706137774009316470178
:1067C000B857370690FF7D16718F558FC166558F6C
:1067D000B8D723A8E712094723AAE7121307704482
:1067E0002391E700938581891386451393850513CB
:1067F0005D45EF10A04D854763FEA70E9387818905
:1068000003A74711050723AAE7109387818983A768
:10681000471163E29708938781891307A044239166
:10682000E700938581891386C510938545065945F0
:10683000EF10605A854763F1A70C93878189FC5359
:1068400093F70770E38607EE138481897C50A18358
:106850009D8B8A07370700201307C749BA978843DB
:10686000EFF0FF82930700707CD09307004523115F
:10687000F400938781891386C710EC535945EF10B4
:1068800040678547E3E6A7EA014545BD93878189CF
:1068900023AA07109DBFB3978700CE9713878189DE
:1068A0002328F7128947232AF712930790422311CE
:1068B000F7004DB59387818903A747114A9703478E
:1068C0000700D8CF5DBD13878189832747118607CD
:1068D000CA9783D707005CCF4DB51387818983277B
:1068E00047118A07CA979C435CCF41BD0145B1B5AA
:1068F0000145A1B5014591B5014581B593878189D0
:1069000003A7871318C183A7C7139CC182809387ED
:10691000818923AE0712372700081307871123AC9C
:10692000E7128280411106C6938781892390070070
:106930002391070023A807109387818983A7071154
:106940000D476361F70213878189139617003E96FE
:1069500093162600BA96154623A0C6148507232849
:10696000F710D9BF9387818923A8071021A89386A0
:1069700081891387770112073697154610C385075B
:1069800023A8F6109387818983A707117D47E370B9
:10699000F7FEB53FEF102042B2404101828093875D
:1069A000818903A5C7118280411106C622C426C26F
:1069B0002A8483D781891307801A6385E70C63785B
:1069C000F7041307101B638EE710637DF70E1307A0
:1069D000701B6382E7221307A01B6392E702938573
:1069E00081891386C510F1051145EF10C03E85471A
:1069F00063F0A72493878189DC4F2320F408239C2C
:106A000001880D45B240224492444101828013071F
:106A1000F0186382E712637EF70813073019638862
:106A2000E7141307C019E39CE7FC9385818913865B
:106A30004513938505131145EF104029854763FFE2
:106A4000A71C9387818903A70711050723A8E710CF
:106A50009387818903A70711FD4763FBE70A9387A3
:106A6000818937072200B8D71307107B2394E706E4
:106A7000B85723A8E712094723AAE7121307801A79
:106A80002390E70093858189138645139385051329
:106A90005D45EF10A023854763F4A718938781898C
:106AA00083A74713638E07101307B01A239CE1884E
:106AB00031A8B1F72320050093878189054723A8D2
:106AC000E71079B71307B01AE39BE7F2EF10800ED7
:106AD000854763F9A714FD577CDC1307101B239C23
:106AE000E188938581891386C510938545065945AC
:106AF000EF10602E854763F9A71293878189FC53B5
:106B000093F70770E1E71307A01B239CE188C1BD41
:106B100093878189B7062200B4D785663697239478
:106B2000E706B85723A8E712094723AAE712130775
:106B3000F0182390E7009385818913864513938588
:106B400005135D45EF108018854763F5A70C938703
:106B5000818983A707110547637CF7021387818921
:106B60000327471331C313073019239CE188EF1023
:106B70006004854763F2A70A9387818983A7071179
:106B8000370700407D17BA978A07A2977D5798C3A9
:106B90009387818923A80712054723AAE7121307C1
:106BA000C0192390E70051B5370700407D17BA9709
:106BB0008A07A297138781890327071398C3C9BF40
:106BC0009387818983A707137CDC01BF9384818924
:106BD000FC50A1839D8B8A07370700201307C74904
:106BE000BA978843EFF0AFCA93070070FCD09307C1
:106BF000701B2390F400938781891386C710EC5390
:106C00005945EF10002F854763F2A702FD57232057
:106C1000F408F5B30145FDB30145EDB30145DDB31E
:106C20000145CDB30145F9BB0145E9BB0145D9BBE0
:106C30000145C9BB411106C622C42A8483D7818974
:106C40001307F01C6388E7021307101D6385E7062E
:106C500081CB239C01880D45B240224441018280B2
:106C600093878189054723A8E7101DA81307F01C07
:106C7000239CE1889387818903A707119317270035
:106C8000A2978565BA958843EFF00FD4854763FFD7
:106C9000A7029387818903A70711050723A8E71097
:106CA0009387818903A70711FD47E3F1E7FC1307E9
:106CB000101D239CE1889305107B03250408EFF049
:106CC000AFD08547E3E7A7F8014579B7014569B734
:106CD000411106C622C42A8483D781891307E01D87
:106CE0006389E7086375F7021307201E6386E70AC6
:106CF0001307401E6388E70C1307001E638CE7042C
:106D0000239C01880D45B24022444101828099CFE5
:106D10001307C01DE396E7FE8567BE952285EFF059
:106D20000FB88547E3EEA7FC0145F1BFFD4763C7F8
:106D3000B7001307C01D239CE188F9BF9307000229
:106D40006385F5029307000463CFB7021307001EA3
:106D5000239CE1888567FD17BE952285EFF02FB44F
:106D60008547E3EFA7F8014579BF1307E01D239C92
:106D7000E1889305107B2285EFF06FB28547E3E150
:106D8000A7F8014549B785679387070463C0B70231
:106D90001307201E239CE1889385F5FB2285EFF0E5
:106DA0000FB08547E3EEA7F40145B1BF8567938730
:106DB00017046385F500FD571CC199B71307401EE2
:106DC000239CE1889305007B138581891305851138
:106DD000EFF0EFAC854763F9A7009387818983A71C
:106DE00087118D8B1CC029BF014531BF411106C6DB
:106DF00022C42A8483D781891307701F6387E70819
:106E00006362F7021307301F638BE7041307501FF9
:106E1000638CE70895CF239C01880D45B24022443E
:106E2000410182801307B01F638DE70A1307D01F4B
:106E30006381E70E1307901FE39FE7FC9385F5FB43
:106E40002285EFF06FB88547E3E7A7FC0145F9B766
:106E5000FD4763C0B7021307301F239CE188856795
:106E6000BE952285EFF04FB68547E3E6A7FA0145C8
:106E700075B7930700026385F5029307000463CF9B
:106E8000B7021307701F239CE1888567FD17BE9525
:106E90002285EFF06FB38547E3EFA7F60145BDBF4D
:106EA0001307501F239CE1889305107B2285EFF088
:106EB000AFB18547E3E1A7F601458DB785679387B5
:106EC000070463C7B7001307901F239CE188BDB771
:106ED000856793871704E390F5F41307B01F239C8D
:106EE000E1889305007B1385818913058511EFF0F7
:106EF0000F9B854763FCA702938781890D8803A7B1
:106F00008711719B598C23AC87101307D01F2390D6
:106F1000E7009305007B9387818903A58711EFF034
:106F2000AFAA8547E3E9A7EE0145CDBD0145FDB513
:106F3000411106C683D781891307B0206386E70411
:106F40006376F7021307D0206386E7061307F02065
:106F50006398E7008146EFF0AFD6854763FAA7064E
:106F6000239C01880D45B24041018280F5FB937757
:106F7000350085E793F735008DE39377360091EF81
:106F80001307B020239CE18889460982EFF04FD394
:106F90008547E3E7A7FC0145F9B79377150085E737
:106FA00093F715008DE39377160091EF1307D02028
:106FB000239CE18885460582EFF08FD08547E3E189
:106FC000A7FA01454DB71307F020239CE18859B774
:106FD000014551BF411106C683D781891307B021EE
:106FE0006386E7046376F7021307D0216386E7061A
:106FF0001307F0216398E7008146EFF06FEF8547B4
:1070000063FAA706239C01880D45B24041018280A6
:10701000F5FB9377350085E793F735008DE393779C
:10702000360091EF1307B021239CE188894609823D
:10703000EFF00FEC8547E3E7A7FC0145F9B793773D
:10704000150085E793F715008DE39377160091EF10
:107050001307D021239CE18885460582EFF04FE994
:107060008547E3E1A7FA01454DB71307F021239CBB
:10707000E18859B7014551BF411106C622C483D7E3
:1070800081891307D0236386E7106362F702130731
:107090000023638FE708130750236386E70CADCB0B
:1070A000239C01880D45B240224441018280130790
:1070B00030246385E70213070025638AE71213076C
:1070C0001024E39FE7FC138581891105EF30203AF6
:1070D000630E051413073024239CE188938581896E
:1070E0001386C510938505054545EF00D04E8547AD
:1070F00063F0A71493878189BC4B93F70720E9E3DA
:107100009387818903A70711050723A8E7104DA0DE
:1071100013878189B707008093E79700B70600209F
:10712000D58F93E727007CC7930700232310F70030
:10713000938781891386C710EC474145EF00705B48
:10714000854763F1A70E0145EFE00FE213848189C3
:10715000E1659385056A13054400EF30202F9307FE
:1071600050232310F400138581891105EF3020305E
:1071700019E101450DBF0545EFE00FDF93878189D8
:107180003707008013679700F8C71307D0232390B1
:10719000E700938781891386C710EC474145EF00CC
:1071A0005055854763F2A7089387818923A8071064
:1071B0009387818903A707119307300663F6E704D5
:1071C000938781893707008013675700F8C7BC4B46
:1071D0001397C7006359070093878189F847B7065B
:1071E0000010558FF8C713070025239CE18893876B
:1071F00081891386C710EC474145EF00904F8547C2
:10720000E3E0A7EA014545B5138481898965938543
:10721000057113054400EF306023930710242310F9
:10722000F40055B5014541B50145B5BD0145A5BDC4
:10723000014595BD83D7818989CB1307D02563810B
:10724000E702239C01880D45828093878189370757
:10725000008013671700F8C71307D0252390E700B5
:10726000411106C6938781891386C710EC474145B3
:10727000EF003048854763F8A700239C01880D453F
:10728000B240410182800145E5BF411106C622C4DA
:1072900026C22A8483D781891307C0266384E70620
:1072A0006376F7021307702A6382E7181307902AA0
:1072B0006389E71A1307B0286380E70A239C0188D3
:1072C0000D45B2402244924441018280A5CB130770
:1072D0009026E395E7FE938581891386C5109385F3
:1072E00005054545EF00302F854763F7A7249387B1
:1072F0008189BC4B93F70720638D07221307C026B3
:10730000239CE1889305007B1385818913058511F2
:10731000EFE0FFD8854763F3A7229387818983A78E
:10732000871193F7071C13070004638EE700130708
:107330000008638DE70099471CC049B713079026E2
:10734000239CE18849BF89471CC08DBF99471CC059
:107350001307B028239CE1889305107B138581894E
:107360001305C512EFE0BFD3854763FBA71C9387C6
:10737000818923A8071031A08507138781892328D5
:10738000F7109387818983A707110D47636FF70271
:1073900093961700BE96139626001387818932971D
:1073A000832607140547E399E6FC13878189139622
:1073B00017003E9693162600BA9683A64614032716
:1073C000C712E39BE6FA85471CC018409947E317AC
:1073D000F7EE9387818923A8071031A085071387CB
:1073E00081892328F7109387818983A707110D4787
:1073F0006367F70293961700BE96139626001387CD
:10740000818932970327071489466301D70C8D467B
:107410006300D70C9146E313D7FC854711A0814741
:10742000E38E07E81307702A239CE188138581897E
:10743000854611468325C51213050537EFF04F88A1
:10744000854763F1A71093848189138684379385D8
:10745000443703A50437EFE0BF8F9307902A2390AA
:10746000F4009387818983A547378567BE95130507
:107470004400EFE0DFC2854763F8A70C938781895A
:1074800083A787375840BA975CC07D57E388E7E207
:107490009387818923A807109387818983A7071180
:1074A0000D47E36DF7E04C4093961700BE96139698
:1074B000260013878189329703274714638CE500E0
:1074C0008507138781892328F710F9B7854789BF76
:1074D0008547B9B793878189B29703A7071489476E
:1074E0006303F7049387818983A607111397160016
:1074F000369793162700B69703A707148D4763079F
:10750000F7029387818983A6071113971600369790
:1075100093162700B69703A707149147E310F7DAED
:1075200095471CC061BB8D471CC06DBF91471CC0F7
:10753000C9BF2320040059B3014561B3014551B3CC
:10754000014541B30145B5BB0145A5BB411106C687
:1075500083D781891307E02C6382E704637BF702FA
:107560001307002D6382E7061307502D639DE70084
:10757000938781891386C710EC474145EF00701748
:10758000854763FEA706239C01880D45B240410153
:107590008280F5FB1307E02C239CE1889305007B98
:1075A0001385818913058511EFE07FAF854763F46B
:1075B000A7049387818903A787116D9B23ACE710EC
:1075C0001307002D2390E7009305007B93878189A3
:1075D00003A58711EFE05FBF854763F0A70293879C
:1075E00081893707004013671700F8C71307502D2C
:1075F0002390E700B5BF014551BF014541BF01459B
:1076000071B7411106C683D781891307F02D6382B4
:10761000E704637BF7021307102E6383E706130763
:10762000602E639DE700938781891386C710EC471E
:107630004145EF00100C854763FFA706239C018896
:107640000D45B24041018280F5FB1307F02D239CCC
:10765000E1889305007B1385818913058511EFE08F
:107660001FA4854763F5A7049387818903A7871122
:107670001367470023ACE7101307102E2390E70091
:107680009305007B9387818903A58711EFE0DFB322
:10769000854763F0A7029387818937070040136706
:1076A0001700F8C71307602E2390E700ADBF014510
:1076B00049BF014579B7014569B7797106D622D42A
:1076C00026D24AD04ECEAE89B2843689E577890774
:1076D0002317F100B7071000938737073EC483D7FD
:1076E00081891307F02F6387E7062A846378F702FE
:1076F0001307A0336387E71C1307B0336382E71EC9
:10770000130700316389E714239C01880D45B250AB
:10771000225492540259F24945618280B5CB130735
:10772000C02FE393E7FE1385818983270511DD07C9
:1077300092073E95310589476387F40A09468546D5
:10774000CE85EFE0FFD7854763F1A7201307F02F21
:10775000239CE1888947638AF40828008947638964
:10776000F40809468546CE85EFE09FF8854763F02B
:10777000A71E9387818903A7071193070002631A45
:10778000F718B9472320F900239C0188094541B720
:1077900035E19387818923A807109387818983A77F
:1077A00007117D47E367F7FC1387770193164700BE
:1077B000138781893697144315476388E600850748
:1077C000138781892328F710C9BF13878189DD07B3
:1077D0009207BA9780C323A2370184C79307C02FAB
:1077E0002310F70089B7054699BF1305E100BDB71F
:1077F00005468DBF9387818923A8071093878189C8
:1078000083A707110D47636FF70E139717003E9775
:107810009316270013878189369783260714154707
:107820006388E6008507138781892328F710F9B755
:1078300093868189139717003E970A07369723206E
:107840008714232237152324971423A2F6129307B3
:1078500000312390F6009305007A9387818903A570
:107860004712EFE07F96854763F5A70E371700288C
:10787000938781891367870523A4E7128947630DDE
:10788000F40863F187028D476301F40A9147631698
:10789000F4029387818903A787121367370023A413
:1078A000E71221A88547631AF4009387818903A70B
:1078B00087121367470023A4E7121307A033239C02
:1078C000E1889305107A9387818903A58712EFE0F9
:1078D000BF8F854763F1A7081307B033239CE18866
:1078E0009387818983A647121397160036970A0754
:1078F000BA979305207A03A54714EFE0FF8C8547DC
:1079000063FDA7049387818903A707119147630744
:10791000F70223200900CDBB9387818903A7871233
:107920001367270023A4E71249BF9387818903A720
:1079300087121367170023A4E71241B7B947232022
:10794000F900239C01880945D9B30145C9B3014514
:107950007DBB01456DBB01455DBB01454DBB411183
:1079600006C622C4368483D78189130760356380B5
:10797000E70C637FF704130780366386E716130767
:1079800090366390E7049305107A0145EFE0DF83BA
:10799000854763F4A7189387818983A607111397F6
:1079A0001600369793162700B697154723A0E714BD
:1079B0009387818903A7071191476306F714232052
:1079C0000400239C01880D45B2402244410182807D
:1079D000EDFB5DE59387818923A8071001A8054683
:1079E0009DA08507138781892328F71093878189B4
:1079F00083A707117D476367F706138777019316FF
:107A000047001387818936971843E31CA7FC138727
:107A1000818936975843E316B7FC138781893697D7
:107A20001847E310C7FC13076035239CE1881385D2
:107A3000818983270511DD0792073E953105894726
:107A4000E30FF6F809468546EFE09FCA854763F2E3
:107A5000A70C9387818903A707115D071207BA97BF
:107A6000154798C39387818903A7071193070002DD
:107A7000E317F7F4B9471CC0239C01880945A9B74F
:107A80009387818923A8071031A0850713878189EF
:107A90002328F7109387818983A707110D47E3698E
:107AA000F7F093961700BE961398260013878189E6
:107AB000429703270714E31AA7FC1387818942978B
:107AC00003274714E313B7FC1387818942970327E1
:107AD0008714E31CC7FA138781892322F7129307BF
:107AE00080362310F7009305007A9387818903A5D8
:107AF0004712EFE06FED854763FFA700130790364D
:107B0000239CE18849B5B9471CC0239C01880945DD
:107B100065BD014555BD014545BD014575B54111E1
:107B200006C6938741C123900700238A0700EFD040
:107B30001FC8EFE0CF93B24041018280411106C6D9
:107B4000EFD01FC9B2404101828083D741C1B9EF54
:107B5000411106C622C426C2AA84938741C103C725
:107B6000470185476318F702138441C123220400AB
:107B700013060002930544001305C400EFE0AF8133
:107B80005C449CC0239A01C00D45B24022449244FB
:107B900041018280138541C15CC1230AF50015466D
:107BA000930545003105EFE0CF837DBF239A01C0E7
:107BB0000D45828083D741C1A5E3411106C622C489
:107BC000938741C103C74701C1476318F702138474
:107BD00041C1C1675CC01306000293054400130550
:107BE000C400EFD05FFB0345540105E5239A01C0B3
:107BF0000D45B240224441018280138541C15CC1E0
:107C0000230AF5001546930545003105EFD07FFDA9
:107C10007DBFEFE02F8ED9BF239A01C00D45828032
:107C200083D741C189C7239A01C00D458280411184
:107C300006C6EFE02F8C239A01C00D45B2404101EA
:107C4000828083D741C1BDEF411106C622C426C23E
:107C5000AA84938741C103C74701C1476318F7044A
:107C6000138441C12322040013060002930544003B
:107C70001305C400EFD03FF25C449CC0918393F79E
:107C8000F7032301F4009C40B1839D8BA30AF40009
:107C900091C7FD17138741C1A30AF700239A01C0BA
:107CA0000D45B2402244924441018280138541C176
:107CB0005CC1230AF5001546930545003105EFD058
:107CC0005FF279BF239A01C00D45828083D741C1FD
:107CD000639F070C011106CE22CC26CA4AC84EC6A5
:107CE0003289AE84AA89938741C103C7270085479B
:107CF000B397E700FD1763ECA70091CD09C61842C2
:107D00008D4763FEE7000545EFD0BF9601A005450E
:107D1000EFD03F9601A00545EFD0BF9501A0938716
:107D200041C103C74701C5476314F7069C408A0752
:107D3000032709000D8BD98F138441C15CC09C407F
:107D4000F9838A09B3E737011CC4034624001306EC
:107D50002602930544001305C400EFD0DFE303457A
:107D6000540139E1138741C15C478D8B2320F90011
:107D70005C478983184B7A07D98F9CC0239A01C02E
:107D80000D45F2406244D2444249B24905618280C5
:107D9000138541C15CC1230AF500154693054500D2
:107DA0003105EFD01FE459B7EFD0DFF465BF239A58
:107DB00001C00D458280411106C6239601C2EFF035
:107DC0001FD6B24041018280411106C6EFF01FD795
:107DD000B24041018280411106C622C426C2AE844F
:107DE000328483D7C1C2130700046381E708637C30
:107DF000F702130730046384E70C1307B004639C95
:107E0000E700EFF03FDB854763F3A70E09C49387D4
:107E1000C1C2DC471CC0239601C20D45B2402244BA
:107E2000924441018280ADCF1307A003E395E7FEA2
:107E30009385C1C21386C500A105EFF03FE98547D0
:107E400063F1A70A9387C1C223A207009387C1C227
:107E5000D843954763EDE7029387C1C223A4070087
:107E600023A60700130700042390E7009385C1C2EF
:107E70001386C500A1050145EFF05FE5854763F472
:107E8000A7069387C1C2D8478D476306F702938739
:107E9000C1C2DC47B1C31307B0042396E1C295B752
:107EA0009387C1C223A407000547D8C71307A003BF
:107EB0002390E700B5BF130730042396E1C21305F2
:107EC0000002EFF0FFD5854763F1A7029387C1C297
:107ED000D8430507D8C39DBF9387C1C29C479CC0A8
:107EE00035B7014525BF014515BF014505BF014512
:107EF00035B7411106C622C4328483D7C1C21307E5
:107F0000F0056387E704637BF70213074006638588
:107F1000E70613078006639CE700EFF0BFC98547BB
:107F200063F4A70809C49387C1C2DC471CC0239629
:107F300001C20D45B240224441018280EDFB93878E
:107F4000C1C28CC70947D8C71307F0052390E700C3
:107F50009385C1C21386C500A105EFF03FD78547C1
:107F600063F0A7049387C1C223A4070023A60700D8
:107F7000130740062390E7009385C1C21386C5000E
:107F8000A1050145EFF09FD4854763FDA7009387C6
:107F9000C1C2DC47C1DB130780062396E1C2B5BF2F
:107FA000014549BF014579B7014569B7411106C689
:107FB000EFE05F97239E01C2B2404101828083D7E8
:107FC000C1C389CB1307D006638AE700239E01C291
:107FD0000D4582801307D006239EE1C2411106C6DB
:107FE00022C42A84EFD05FEA854763F9A7021C40C8
:107FF00081CB239E01C20D45B240224441018280C3
:10800000EFE0FF99B75700109387D763E303F5FEBE
:1080100089471CC0239E01C20945F9BF0145E9BF3C
:10802000411106C622C42A8483D7C1C3130700089E
:10803000638AE7086373F708130760086380E70A39
:108040001307D0086394E7061146B7F5FF1F938521
:10805000057E1385C1C33105EFE09FED854763FAC7
:10806000A70C9387C1C3DC479386F7FF75576367F7
:10807000D70AC207C1831397A7009387C1C323A060
:10808000070223A20702B706000894D7054690DB33
:10809000D4DB98DF13060040D0DF23A00704BA9694
:1080A000F4C3B70600F83387E640B8C7239E01C281
:1080B0000D45B240224441018280EDFB13070008C8
:1080C000239EE1C22285EFE0AFA1854763FFA704AD
:1080D0001C409DEB13076008239EE1C21146B725A3
:1080E0000240F1051385C1C33105EFE07FE4854708
:1080F00063FFA7029387C1C3DC47898B91EB13070A
:10810000D008239EE1C289B7239E01C2094555B715
:1081100091471CC0239E01C2094561BF9307F00F20
:108120001CC0239E01C2094569B7014559B70145E5
:1081300049B70145BDBF83D7C1C389CB1307B00A77
:10814000638AE700239E01C20D4582801307B00AAF
:10815000239EE1C2411106C6EFE08FAA854763F86E
:10816000A700239E01C20D45B24041018280014516
:10817000E5BF411106C6EFD0BFF0B2404101828099
:10818000411106C622C426C24AC0AA842E8932845E
:1081900083D7C1C31307600D6389E70C637DF706BE
:1081A0001307F00E6382E7046368F7241307C00D1A
:1081B0006383E71E6376F71A1307000E638CE73AB2
:1081C0001307E00E6395E70E1146B7250240C1057F
:1081D0001385C1C33105EFE0FFDF854763FDA7428B
:1081E0001307F00E239EE1C21146B7250240D105C8
:1081F0001385C1C35105EFE0FFDD854763FFA7404D
:108200009387C1C3D84713670704D8C71307100F54
:108210002390E7001DA41307100C638EE730637EE4
:10822000F7061307A00C638FE70C637BF7081307AF
:10823000F00C638FE70E1307200D639AE7061146D3
:10824000B71502401385C1C33105EFE0BFD885479C
:1082500063F9A73A9387C1C3984B719B13672700B3
:1082600098CB1307600D2390E7001146B715024025
:1082700091051385C1C34105EFE0DFD5854763F460
:10828000A7389387C1C33707674513073712D8C785
:108290001307A00D2390E700C1A81307C00B63824A
:1082A000E7241307D00B638DE72463880722239EFE
:1082B00001C20D45B24022449244024941018280EC
:1082C0001307600CE395E7FE1146B71502409105D0
:1082D0001385C1C34105EFE0FFCF854763FDA7309C
:1082E0009387C1C3DC47139767006358070213875E
:1082F000C1C3B70600FFFD16F58F5CC79307A00C3E
:108300002310F7001146B71502401385C1C331058C
:10831000EFE05FCC854763F2A72E9387C1C3370791
:108320002C201307074098CB1307F00C2390E7008D
:108330001146B715024091051385C1C34105EFE011
:108340007FC9854763FDA72A9387C1C3D847B7066E
:108350000001558FD8C71307200D2390E700C5B53E
:108360001307A00DE395E7F41146B72502409105E8
:108370001385C1C33105EFE0FFC5854763F7A72823
:108380009387C1C33797EFCD1307B79AD8C71307A1
:10839000C00D2390E7001146B725024091051385D3
:1083A000C1C33105EFE01FC3854763F2A72693875A
:1083B000C1C323AE07009387C1C3D84F954763D786
:1083C000E71A9387C1C3DC4793F70708639D071C2F
:1083D0009387C1C3C4CBCA9484CF9387C1C3D84BFE
:1083E0009C4F6368F71C9387C1C323A6070013073C
:1083F000E0102390E70039A81307800F6388E70691
:108400006379F70213074010638BE70A1307E01044
:10841000E39FE7E81146B7250240C1051385C1C3B4
:108420003105EFE03FBB854763FFA71E2320040013
:10843000BDBD1307100FE39CE7E61146B7250240C8
:10844000C1051385C1C33105EFE0DFB8854763F887
:10845000A71CB72509009385057C1385C1C31105A9
:10846000EF10D07E1307800F239EE1C21146B7257F
:108470000240B1051385C1C33105EFE07FAB8547ED
:1084800063F1A71A1385C1C31105EF10507E11E5E2
:108490009387C1C3DC47858BF1F79387C1C3DC4762
:1084A00013F7170063100712C18B638907129387B4
:1084B000C1C34147D8C7130740102390E7001146B6
:1084C000B7250240B1051385C1C33105EFE09FB068
:1084D000854763EFA70E0145F1BB1307C00B239E31
:1084E000E1C21146B71502401385C1C33105EFE063
:1084F0003FA4854763FBA70E1307D00B239EE1C261
:108500001146B715024091051385C1C34105EFE03F
:108510003FA2854763FDA70C9387C1C3DC4713F7D0
:1085200027000DE71387C1C393E717005CC79307C4
:10853000100C2310F7001146B71502401385C1C374
:108540003105EFE03FA9854763F5A70A9387C1C3CB
:108550009C4B13F7C700E30507D81387C1C3F19BF2
:108560001CCB9307600C2310F700B9BB1307000E58
:10857000239EE1C21146B7250240C1051385C1C340
:108580003105EFE0FF9A854763F5A7089387C1C3DC
:10859000DC4793F70708E38607E29387C1C3D84F08
:1085A0000507D8CF09BD85471CC0239E01C20945D8
:1085B00011B39387C1C30947D8C71307E00E2390AF
:1085C000E70019B189471CC0239E01C20945DDB1EE
:1085D0008D471CC0239E01C20945E9B99387C1C3D9
:1085E000D84B13070740D8CBCDBB0145E1B10145BE
:1085F000D1B10145C1B1014575B9014565B9014523
:1086000055B9014545B9014575B1014565B101450A
:1086100055B1014545B1014571B9014561B9014502
:1086200051B9014541B9014571B1011106CE22CCC4
:1086300026CA4AC84EC62A89AE893284B68483D7F0
:10864000C1C31307E011638FE7046378F7021307D0
:1086500070126381E70A1307E0146388E70E1307BB
:108660000012638DE704239E01C20D45F24062446F
:10867000D2444249B24905618280D9CB1307B01177
:10868000E393E7FE1146B7250240C1051385C1C338
:108690003105EFE03F94854763F8A70C1307E0111D
:1086A000239EE1C24E86CA852285EFE0BF928547B0
:1086B00063FEA70A13070012239EE1C21146B725E5
:1086C0000240B1051385C1C33105EFE07F868547C0
:1086D00063F0A70A9387C1C3DC4713F7170031E3A0
:1086E000918BA1CF9387C1C31147D8C713077012CD
:1086F0002390E7001146B7250240B1051385C1C399
:108700003105EFE03F8D854763E3A7020145B9BF1F
:108710009387C1C30547D8C71307B0112390E7005B
:1087200095B789479CC0239E01C2094581B78D47F3
:108730009CC0239E01C2094515BF9387C1C323A6D0
:1087400007001307E0142390E7001146B725024005
:10875000C1051385C1C33105EFE0DF87854763FBA2
:10876000A70023A0040001B7014509B70145FDBDDD
:108770000145EDBD0145DDBD411106C683D7C1C32D
:108780001307B0156387E704637BF7021307E0154F
:108790006386E70613071016639DE7001146B715B9
:1087A00002401385C1C33105EFE0DF82854763F1E5
:1087B000A708239E01C20D45B24041018280F5FB0E
:1087C0009387C1C313070008D8C71307B0152390B8
:1087D000E7001146B7250240C1051385C1C3310525
:1087E000EFE04FFF854763F1A7049387C1C33707C5
:1087F0002C2098CB1307E0152390E7001146B715FE
:10880000024091051385C1C34105EFE0AFFC8547E8
:1088100063FEA7009387C1C313073008D8C71307A7
:1088200010162390E7009DBF014579B7014569B750
:10883000014559B7372500081305051B82801385AC
:10884000C1C31305050282800D458280814701471F
:1088500063F9B700B306F50083C6060036978507AF
:10886000C5BF1375F70F82809387C1C823A0070087
:108870007D5798C7D8C723A80700238A0700938786
:10888000C10A05472380E700A380070023A2070051
:10889000828015A01387C1C83E97834657011307EE
:1088A00040026396E6021387C1C81CC70DA0850766
:1088B0001387C1C81CCB1387C1C81C4B184363FB6B
:1088C000E7021387C1C814477D57E385E6FC138789
:1088D000C1C854477D57E39CE6FC1387C1C83E9747
:1088E0008346570113073002E393E6FC1387C1C8A0
:1088F0005CC775BF9387C1C89C4763C70700938651
:10890000C1C8D4466345D0028547631EF7029387EA
:10891000C1C803C757018D476319F7021385C1C842
:108920008547230AF50085475CC15505828013857C
:10893000C1C80547230AE5009D8EFD1654C1C50731
:108940003E9515058280014582800145828093878E
:10895000C1C8C84382809387C1C8238A070023A067
:10896000070023A207007D5798C7D8C723A8070090
:1089700082809387C1C883C74701B9E383A6C1C872
:1089800013078040158F6374B7003E8582804111C4
:1089900006C622C426C22E84AA859384C1C8C106F5
:1089A000A696228613855600EF10307A8C40A29549
:1089B0008CC085473E85B24022449244410182806A
:1089C0008147E1B783C7C10A89C71385C10A390541
:1089D0008280014582809387C10A23800700C8C333
:1089E00093F715008DC79387C10A13074002A3862A
:1089F000E70083C7170099EF9387C10A1307B002F6
:108A00002386E70023A4070013072500D8C389891C
:108A100091E982809387C10A054798C7130715001B
:108A2000D8C3F5B7411106C622C426C24AC0AA85DA
:108A30001384C10A032944000444B3079900A29790
:108A4000130730022386E7000509232224011305BA
:108A5000E400EFF0BFDFCA94A294AA86372600088C
:108A60001306C61B8D451385C400EF20E0035C4050
:108A700089075CC0B240224492440249410182808D
:108A800083C7C10A89EB9387C10AD84318C18847B5
:108A90003E9531058280014582809387C10A23A2D9
:108AA000070005472380E70082809387C10AA380DF
:108AB000A7008280814629A8130777052380E50057
:108AC00035A093877705A380F50089050505850600
:108AD00063F6C6028347050013D74700BD8B2548C0
:108AE000E36CE8FC130707032380E5002547E36AEE
:108AF000F7FC93870703A380F500C1BF82800111B3
:108B000006CE2306A10093578500A306F1009357D4
:108B100005012307F1006181A307A1001146680048
:108B2000EFF05FF9F2400561828081461DA81308CD
:108B300060046369F804938797FC93F7F70F2A970B
:108B400003471700130890036363E804130707FD46
:108B50001377F70F92073388D500D98F2300F800D9
:108B6000850663F4C60413971600B307E50083C7B0
:108B7000070013089003E36CF8FA938707FD93F757
:108B8000F70F75BF938797FA93F7F70F4DBF130849
:108B900060046367E800130797FC1377F70F5DBF66
:108BA000130797FA1377F70F75B78280011106CE76
:108BB00022CC2E8411466C00EFF03FF78347C100B2
:108BC0000347D1002207D98F0347E1004207D98F1D
:108BD0000347F1006207D98F1CC0F240624405616F
:108BE000828081488147814639A03388D50023009F
:108BF000E8008506850763F6C7023307F5000347DB
:108C000007001308D007630C0701E38008FE3388D0
:108C1000D500134707022300E8008148D9BF8548E3
:108C2000D1BF36858280411106C69387014C238AC5
:108C3000A700EFC03FA3B24041018280411106C6A8
:108C40008D450145EFF03FD9B2404101828041118D
:108C500006C613060040B73500089385058E938736
:108C6000014C884BEF10F0758D450945EFF0BFD6EC
:108C7000B24041018280411106C622C41384014CD6
:108C8000AA86373600081306868D930500400848EB
:108C9000EF1090610848EF10F06E8D45EFF0BFD3F4
:108CA000B240224441018280411106C622C413848D
:108CB000014C231004002311040023120400231389
:108CC00004000145EFF03FF6A30A0400B24022443D
:108CD00041018280011106CE9387014C8847340000
:108CE0007000B7250008938545537D05EF10B062ED
:108CF00022479307004063F3E7003EC4EFD0CF84E0
:108D0000B2471D8DA24763EEA7022AC49387014C88
:108D10009C4B1307C0062380E700EFD04F82938758
:108D2000014C9C4B2246B245AA9513851700EF10C3
:108D300050698D4522450505EFF0FFC9F2400561F8
:108D400082809387014C9C4B1307D0062380E70059
:108D5000E9B7011106CE22CC26CA4AC84EC6EFF0AA
:108D6000BFAE2A89EFF0BFADAA849389014C394682
:108D7000B72500089385856503A50901EF10F03C30
:108D8000354423A809421DA8B72600089386066526
:108D9000A9A89387014C884B372600081306066D57
:108DA00093050040818D2295EF10105009049387A0
:108DB000014C03A70743050723A8E7429387014C0B
:108DC00003A70743637627079387014C884B2295B7
:108DD00093050040818D1207269714438547E3854C
:108DE000F6FAB72600089386C6641C475843372610
:108DF000000813068666EF10304B2A949387014CC7
:108E000083A707439207A69794430547E393E6F8A1
:108E10001387014C084BD447372600081306866990
:108E200093050040818D2295EF1010482A9441B798
:108E30009387014C884B372600081306466D93052F
:108E40000040818D2295EF1030468D451305D400EA
:108E5000EFF07FB8F2406244D2444249B249056122
:108E60008280397106DE22DC26DA4AD8B72700086C
:108E700003A3475C9387475C83A8470003A8870048
:108E8000C8478C4BD04B944FD84F1AC046C242C4EF
:108E90002AC62EC832CA36CC3ACE83C70702230070
:108EA000F1029387014C83D747001307A017638211
:108EB000E7086374F702130720186383E70C1307AE
:108EC000F0186398E70CEFF0FFAF9387014C88CB65
:108ED00063040518EFF0BFD76DA8C5EF1305F102C5
:108EE000EF10405231CD9387014C9C4B1307F00497
:108EF0002380E70001449387014C8C4B93171400A7
:108F000085070546BE951305F102EFF0BFBA0504CB
:108F10001305F102EF10004F79FD131514008D4574
:108F20000505EFF05FAB9387014C1307A017239261
:108F3000E700EFF03FA99387014C88CB630C051045
:108F40001384014C50446916058210D408449304DC
:108F5000C402A6851905EFF05FBD1C543E9423069C
:108F600004021546B7250008938585582685EF101D
:108F700090421DE99387014C130720182392E700C4
:108F8000EFE08F8F854763E4A700014501A8EFF06C
:108F90001FCC9387014C239207000D45F250625479
:108FA000D2544259216182801146B7250008938529
:108FB00005591385014C1305C502EF10D03D35C985
:108FC0002946B7250008938585591385014C13055B
:108FD000C502EF10503C2DE14C102810EFD01F922D
:108FE0001384014C1309C4021257A25637260008F5
:108FF0001306465A930500404A85EF10F02A4A8529
:10900000EF105038AA841C481307F0042380E700AF
:109010000C482A8685054A85EFF0DFA913951400D0
:109020008D450505EFF03F9B9307F0182312F400E0
:1090300059BDEFF0DFC1B1BF130600029387014CA9
:109040008C4B0A85EFF01FA78D4513050004EFF048
:109050009F9881B7014599B7014589B79387014C1E
:1090600083D7270095EF411106C63D46B725000876
:10907000938505529387014C8847EF10D03111ED4D
:10908000EFF0FFBC0545EFF05FA29387014C239101
:1090900007000D45B24041018280EFF03FBAF5B7BD
:1090A0009387014C239107000D4582809387014CE3
:1090B00083D72700CDEF011106CE22CC9387014C38
:1090C000884703441500930770066302F402930770
:1090D0007004630EF4009307D006630AF40093074C
:1090E000D0046306F40093073006631FF406700093
:1090F000B72500089385C5510905EF10D021EFF081
:109100001FB50317C100930770066303F4029307AA
:109110007004630CF4029307D006630DF402930706
:10912000D004630EF4029387014C2394E74C29A0EA
:109130009387014C2390E74C9387014C23910700C0
:109140000D45F2406244056182809387014C239172
:10915000E74CDDB79387014C2392E74CF1BF93872F
:10916000014C2393E74CC9BFEFF05FADF1B7938794
:10917000014C239107000D4582809387014C83D7D2
:10918000270099C79387014C239107000D458280E2
:10919000411106C613060040B72500089385856473
:1091A0009387014C884BEF10D0218D450D45EFF092
:1091B0009F829387014C239107000D45B2404101E6
:1091C00082809387014C83D7270099CB1307B01E69
:1091D000638EE7009387014C239107000D45828041
:1091E0009387014C1307B01E2391E700411106C677
:1091F00022C41385014C13054543EFD0EFFA854790
:1092000063F4A70401449307000263C187029387B4
:10921000014C8C4B931634001307C4100A07BA97FD
:10922000B695C843EFF0BF8D0504F1BF8D4513051A
:109230008010EFF04FFA9387014C239107000D4502
:10924000B2402244410182800145DDBF411106C682
:1092500022C49387014C83D7270091CF1307502056
:109260006386E7049387014C239107000D45B240C4
:1092700022444101828001449307000263C28702B5
:109280009385014C88459317340085071307C41054
:109290000A07BA9591053E95EFF05F910504E9BF85
:1092A0009387014C130750202391E7001385014C4D
:1092B00013054543EFD01F98854763E4A700014598
:1092C0007DB7EFF0DF9879BF411106C622C49387BE
:1092D000014C83D7270091CF13077021638BE702DE
:1092E0009387014C239107000D45B2402244410170
:1092F00082801384014C08441306C44BB725000830
:109300009385C5510505EF101001930770212311B6
:10931000F4001385014C8325C54B1305854BEFD015
:109320003F9B854763E4A7000145C1B79387014C84
:109330008C4B03A5874BEFF08FFC8D452145EFF05B
:109340008FE979BF411106C622C49387014C83D7A8
:10935000270091CF130710236386E7049387014CFE
:10936000239107000D45B2402244410182801384BD
:10937000014C08441306C44BB72500089385C5511A
:109380000505EF10407908449305D0030505EF105B
:10939000C07D9305844B0505EFF05F819307102393
:1093A0002311F4009387014C83A5C74B03A5874B7A
:1093B000EFD0DFA3854763E4A70001456DB7EFF069
:1093C0001F8969BF011106CE22CC26CA4AC84EC6E3
:1093D0009387014C83D727008DC31307002563892A
:1093E000E7069387014C239107000D45F240624444
:1093F000D2444249B249056182801384014C04443D
:1094000085049305C0022685EF1020769309150088
:1094100013064402372900089305C9512685EF1029
:10942000806F130684029305C9514E85EF10A06E1C
:1094300018549307004063F7E7009387014C130724
:10944000004098D79387014C130700252391E7002C
:109450001385014C10554C511305C502EFD05FAD7B
:10946000854763E4A700014551B71384014C1054AC
:109470000C481305C402EFF0EFE308548D450605D0
:10948000EFF06FD5B9BF411106C622C49387014CD6
:1094900083D7270091CF1307C0266385E7069387FC
:1094A000014C239107000D45B240224441018280C6
:1094B0001384014C08449306840213064402B72522
:1094C0000008938545530505EF10E06408449305B3
:1094D000A0030505EF1060690505185493070040C7
:1094E00063F7E7009387014C1307004098D7138474
:1094F000014C10549305C402EFF02FE39307C026EC
:109500002311F4001385014C10554C511305C5026D
:10951000EFD05FAC854763E4A700014571B7EFF07A
:109520000FF3B5BF411106C622C426C29387014C72
:1095300083D7270099CF1307F028638CE70693871A
:10954000014C239107000D45B24022449244410151
:1095500082801384014C084493068402130644025B
:10956000B7250008938545530505EF10C05A0054F0
:1095700031CC9387014C84479305A00313851400D5
:10958000EF10A05E05059307004063F787009387FF
:10959000014C1307004098D71384014C5044898C28
:1095A00026969305C402EFF0CFE39307F02823112A
:1095B000F4001385014C10554C511305C502EFD032
:1095C0007FA1854763ECA7000145BDBFEFF02FE801
:1095D0009387014C239107000945BDB7EFF02FE7B2
:1095E000B9BF9387014C83D7270099CB1307F02A83
:1095F000638EE7009387014C239107000D4582801D
:109600009387014C1307F02A2391E700411106C606
:10961000EFD0DFF3854763E6A7000145B240410183
:1096200082800545EFF02FE09387014C23910700DE
:109630000D45EDB79387014C83D7270099CB1307CE
:10964000E02B638EE7009387014C239107000D45C3
:1096500082809387014C1307E02B2391E70041118F
:1096600006C6EFD01FFA854763E6A7000145B24062
:10967000410182800545EFF00FDB9387014C239178
:1096800007000D45EDB7011106CE22CC9387014CA2
:1096900083D7270091CF1307602D6384E704938756
:1096A000014C239107000D45F24062440561828020
:1096B0001384014C580034007000B72500089385CE
:1096C00005720844EF102045B2472326F44CA24708
:1096D0002328F44C9247232AF44C9307602D23113E
:1096E000F4009387014C9386874D03A6474D83A5CD
:1096F000074D03A5C74CEFE08FA6854763FDA70084
:109700009387014C03A5874D01E5EFF04FD441BF8E
:10971000EFF06FD669B7014541BF011106CE22CCEB
:109720009387014C83D7270091CF1307202F6384A1
:10973000E7049387014C239107000D45F2406244F2
:10974000056182801384014C580034007000B725F5
:109750000008938505530844EF10E03BB2472326E9
:10976000F44CA2472328F44C9247232AF44C930745
:10977000202F2311F4009387014C9386874D03A675
:10978000474D83A5074D03A5C74CEFD01FF3854771
:1097900063FDA7009387014C03A5874D01E5EFF01A
:1097A0000FCB41BFEFF02FCD69B7014541BF938784
:1097B000014C83D7270099CB13074030638EE70015
:1097C0009387014C239107000D4582809387014CBC
:1097D000130740302391E700411106C6EFD09FA543
:1097E000854763FAA7009387014C239107000D4535
:1097F000B240410182800145E5BF9387014C83D788
:10980000470099CB13076036638EE7009387014CBE
:10981000239207000D4582809387014C1307603621
:109820002392E700411106C6EFE01FF5854763E686
:10983000A7000145B24041018280EFF04FC19387FC
:10984000014C239207000D45F5B7011106CE22CC3D
:109850009387014C83D767001307A03A6382E70818
:109860006379F7041307D03A638FE7081307E03AE8
:10987000639CE70E1385014C13050502EFE04FFAD8
:10988000854763F5A7129387014C9C53D5C30947BD
:109890006385E70E6375F7080D476387E70E114789
:1098A000639BE70E372500081305857DEF00F03236
:1098B00041A0DDEB1305F100EF00D03465FD054557
:1098C000EFB07FD91384014C8547A30AF40001450A
:1098D000EFF06FB5EFE08FED9307A03A2313F4009C
:1098E0001385014C13050502EFE06FED854763FB1F
:1098F000A70A9387014C9C53D9F79387014C130710
:10990000D03A2393E700EFD0FF92854763FEA70884
:109910009387014C1307E03A2393E700A1BF054763
:10992000639BE706372500081305C572EF00F02A90
:109930003735000813058584EF00302A37350008D5
:1099400013058585EF007029373500081305458616
:10995000EF00B028EFE01FEEEF00302837350008A9
:1099600013054587EF0070279387014C2393070069
:109970000D45F240624405618280372500081305D9
:10998000C575EF0090256DB7372500081305457A9A
:10999000EF00B02471BF3735000813058582EF0052
:1099A000D02379B70145F1B70145E1B70145D1B7FA
:1099B000597186D6A2D4B72700089387875E0A8795
:1099C0009386070503A80700C8438C47D047232088
:1099D000070148C30CC750C7C1074107E394D7FE2E
:1099E0008C43D04394470CC350C314C783D7C700DC
:1099F0002316F7009387014C83D7470091CF1307B5
:109A0000F0106380E7049387014C239207000D4513
:109A1000B6502654656182800145EFF00F891384AA
:109A2000014C130600408A850848EF1080190A850A
:109A3000EF1040158D45EFE01FFA9307F010231249
:109A4000F400EFF09FE08547E3EFA7FA0145C9B7BF
:109A5000411106C622C49387014C83D72700130700
:109A6000B00E6382E7041307100F6386E70891CBFB
:109A70009387014C239107000D45B24022444101D8
:109A800082809387014C80472D46B7250008938537
:109A9000C5532285EF10201011ED9387014C130759
:109AA000B00E2391E700EFF0BFF08547E3E2A7FC9B
:109AB0000145E1B77D46B725000893858554228589
:109AC000EF10600D21C15D46B725000893858556CE
:109AD0002285EF10400C15C91946B725000893855B
:109AE00005582285EF10200B05E59387014C1307DD
:109AF000100F2391E700EFF0CFB68547E3EAA7F612
:109B00000145A5BFEFF00F9DA5B7EFF08FA48DB76E
:109B1000EFF0CF92B1BF411106C69387014C83D7B6
:109B200067001307503D6380E7041307B03D63806F
:109B3000E70689CB9387014C239307000D45B2407C
:109B4000410182809387014C83C747018DE793874A
:109B5000014C985385476300F7029387014C130724
:109B6000503D2393E700EFD07F9E854763F0A70425
:109B70000545EFF04F8B9387014C98538547630D54
:109B8000F7009387014C1307B03D2393E700EFE004
:109B90008FDA854763FEA700EFE0AFDD9387014CC6
:109BA000A38A07000145EFB01FAB69B7014541BF6C
:109BB000014571B7411106C69387014C83D7270031
:109BC00089CF1307002A6382E7029387014C239110
:109BD00007000D45B24041018280EFF04F87938727
:109BE000014C1307002A2391E700EFF0DFF28547CD
:109BF000E3EDA7FC0145F9BF011106CE22CC938706
:109C0000014C83D74700130700336384E70413072D
:109C100050336388E70691CB9387014C239207006A
:109C20000D45F2406244056182801384014C084472
:109C300034007000B7250008938545533105EF00C7
:109C4000906DB2475CD0A2471CD493070033231217
:109C5000F4009387014C1386C7428C57C853EFE03A
:109C60002FD2854763F9A7029387014C03A5C7420A
:109C700005C1EFF04F809387014C130750332392B7
:109C8000E700EFF05FE98547E3E8A7F8014551BF3A
:109C9000EFE0FFFB51B7014569B7011106CE22CCB9
:109CA00026CA9387014C83D7470013072035638268
:109CB000E706130770356388E70899CB9387014C53
:109CC000239207000D45F2406244D2440561828030
:109CD0001384014C08447000B72500089385C551D2
:109CE0003105EF005063B2475CD004449305A003F4
:109CF0001385C400EF00706705055044898C2696D3
:109D00009305C402EFE0FFED08D49307203523123A
:109D1000F4009387014C9386C7421386C7028C5781
:109D2000C853EFE09F90854763F9A7029387014CE2
:109D300003A5C74205C1EFE01FF49387014C130749
:109D400070352392E700EFF01FDD8547E3E8A7F6C3
:109D5000014595BFEFE0BFEF95B70145ADB70111E4
:109D600006CE22CC9387014C83D7470091CF1307AF
:109D70002038638CE7049387014C239207000D453C
:109D8000F2406244056182809387014C9C538DC3ED
:109D900001441305F100EF00E06611CD9387014CFB
:109DA0009C4BA2970347F1002380E7000504D5B739
:109DB000EFE0DFE8C9B78D452285EFE0DFC193878B
:109DC000014C130720382392E700EFF0DFD48547DA
:109DD000E3E3A7FA01456DB7411106C622C4938794
:109DE000014C83D72700130750316388E70863715C
:109DF000F702130770316388E70A13079031639302
:109E0000E702EFF0DFF5854763EEA700014505A007
:109E10009DC3130730316397E700EFF0FFDD8547FF
:109E200063FDA70A9387014C239107000D45B240BB
:109E30002244410182809387014C80473146B725F7
:109E400000089385456E2285EF00F05401E9938761
:109E5000014C130730312391E700C1B73146B725D4
:109E600000089385456F2285EF00F05211ED93872E
:109E7000014C130750312391E700EFF01FE28547B3
:109E8000E3E2A7FA014565B72946B725000893859F
:109E900045702285EF00305011ED9387014C130778
:109EA00070312391E700EFF05F958547E3ECA7F66B
:109EB0000145B5BF3D46B72500089385057122854C
:109EC000EF00704D01E99387014C13079031239106
:109ED000E70005BFEFE09FD6B1B7014589BF83D743
:109EE000014C1307500D6368F746011106CE22CCD2
:109EF0008A07372700081307471CBA979C438287B5
:109F00009387014C83C757016393070E1307E00A39
:109F10002390E14CEFE0FF979387014C88C76306DD
:109F20000542EFE0DFA29387014CC8C71307100B6F
:109F30002390E700EFE01FA99387014C88CB6308CB
:109F400005409387014C9C4783C70700A307F10096
:109F5000130710076385E726130710056385E728B5
:109F600013078004638CE7281307F0036383E72A51
:109F700013077006638AE72A130770046381E72CCE
:109F80001307B0066388E72C13073006638FE72CAE
:109F90001307D0066386E72E1307D004638DE72EE0
:109FA000130780056384E73013070007638BE730EE
:109FB000130700056382E732130730076389E7322E
:109FC0001307A0076380E7341307A0056387E7340E
:109FD00013076007639EE7341307500D2390E14C8D
:109FE000EFF09FDF854763E5A71E0145CDAA938764
:109FF000014C83C74701E38B07F01305F1001921DA
:10A0000039C99387014C9C4B1307F0042380E70068
:10A0100001449387014C8C4B931714008507054628
:10A02000BE951305F100EFE0FFA805041305F1004C
:10A03000D12E65F1131514008D450505EFE0BF998C
:10A04000130760082390E14CEFE0DF979387014C02
:10A0500088CB6306052EEFE0DF839387014C88C72A
:10A0600021CDEFE0DF8E9387014CC8C79C4703C723
:10A0700007008D476310F7048547631DF50213073A
:10A08000D0082390E14CEFF08FF2854763FBA72ABD
:10A090000145EFE05FB913060040B735000893852E
:10A0A00005889387014C884BEF00B0318D450D45F5
:10A0B000EFE07F92EFE03F8A9387014C83C747012F
:10A0C000638A0710130760092390E14C1385014C44
:10A0D0006105EFD08F9B854763F7A7269387014CD7
:10A0E0009C4F6389070E0145EFE0FFB39387014C56
:10A0F0009C4F1947638AE7020D476383E7041147C2
:10A10000638DE70415476387E70605476381E70822
:10A110000947638AE7089387014C884BEF00902634
:10A120008D45EFE05F8B7DA013060040B73500083A
:10A13000938545889387014C884BEF009028E1BFB9
:10A140009387014CD44F3736000813068688930551
:10A150000040884BEF0050157DBF9387014CD44FD2
:10A16000373600081306868993050040884BEF00B8
:10A17000B01355B79387014CD44F373600081306F8
:10A18000868A93050040884BEF00101269B71306CA
:10A190000040B73500089385858B9387014C884B29
:10A1A000EF0030228DBF13060040B73500089385BD
:10A1B000858C9387014C884BEF00B020A9BF130713
:10A1C000500B2390E14CEFF0BF88854763F3A7184D
:10A1D000EFE06FF8130770072390E14C0545F2405C
:10A1E0006244056182801307700B2390E14CEFE01D
:10A1F000FFE68547E3EEA7FC0145D5B71307900BB3
:10A200002390E14CEFE09FEA8547E3E3A7FC01459B
:10A21000F9B71307B00B2390E14CEFE01FF6854729
:10A22000E3E8A7FA014565BF1307D00B2390E14C83
:10A23000EFE03FF98547E3EDA7F801454DB7130778
:10A24000F00B2390E14CEFF06F808547E3E2A7F835
:10A25000014571B71307100C2390E14CEFF09F9567
:10A260008547E3E7A7F601459DBF1307300C239010
:10A27000E14CEFF00FB78547E3ECA7F4014585B754
:10A280001307500C2390E14CEFF0CF938547E3E1A7
:10A29000A7F40145A9B71307700C2390E14CEFF028
:10A2A0008F9E8547E3E6A7F2014515BF1307900C83
:10A2B0002390E14CEFF00FA78547E3EBA7F00145B2
:10A2C00039BF1307B00C2390E14CEFE0FFFF854747
:10A2D000E3E0A7F0014521B71307D00C2390E14C30
:10A2E000EFF04F868547E3E5A7EE0145CDBD1307A7
:10A2F000F00C2390E14CEFF0EFB38547E3EAA7ECD5
:10A300000145F1BD1307100D2390E14CEFF0AFB7FD
:10A310008547E3EFA7EA0145D9B51307300D239030
:10A32000E14CEFF08FBF8547E3E4A7EA014545BD67
:10A33000EFE0DF9071BD2390014C0D454DB5014517
:10A3400079BD014569BD014559BD014549BD01457D
:10A3500079B5014569B52390014C0D4582804111C5
:10A3600006C6EFB08F990D20EFA0BFF6EFE0CFCF7C
:10A37000EFE09F93EFB00FA00D20EFA09FF9EFB09B
:10A380008F84EFF0DFB5FDB7B727002093874782B2
:10A3900023A0070023A2070082800D458280B727F3
:10A3A000002083A74782138717009306F00F63D31B
:10A3B000E6000147B726002093864682D442638C8C
:10A3C000E600B726002093864682B6972384A7002E
:10A3D00098C20545828001458280411106C622C48B
:10A3E00026C22A8481440345040019C5EFF03FFBCF
:10A3F00001C505048504C5BF2685B24022449244A8
:10A4000041018280B727002093874782D8439C432D
:10A41000630AF702B7270020938747823E970347D6
:10A4200087002300E500D8430507D8C39307F00F42
:10A4300063DCE700B72700209387478223A2070049
:10A44000054582800145828005458280411106C60E
:10A4500022C42A844CC1EFB08F8408C0B240224489
:10A460004101828058411C41BA971CC18280411130
:10A4700006C622C42A84EFB08F821C401D8D0505BC
:10A480005C4033B5A700B240224441018280000005
:10A4900000000000000000000000000000000000BC
:10A4A00000000000000000000000000000000000AC
:10A4B000000000000000000000000000000000009C
:10A4C0005D7106C012C216C41AC61EC82ACA2ECC96
:10A4D00032CE36D03AD23ED442D646D872DA76DC84
:10A4E0007ADEFEC0F322103496C0F322003096C20A
:10A4F000F322407C96C4732520348A85EFA07FFC2C
:10A50000864273901234964273900230A642739042
:10A51000427C82401242A2423243C2435245E2454B
:10A52000724682561257A2573258C258525EE25EA5
:10A53000725F864F616173002030000000000000F0
:10A540005D7106C012C216C41AC61EC82ACA2ECC15
:10A5500032CE36D03AD23ED442D646D872DA76DC03
:10A560007ADEFEC073D0E87E7350F97E73D0B97E78
:10A57000F390D07E73700430B6427390427CA64252
:10A580007390123496427390223482401242A24257
:10A590003243C2435245E245724682561257A25791
:10A5A0003258C258525EE25E725F864F616173003C
:10A5B0002030B687B2882A832E88639D061463F9FB
:10A5C000C50A4167636EE61AB70700016363F63494
:10A5D00093568601E1471787FFFF1307E730369749
:10A5E00003470700BA97130700021D8F19CB339852
:10A5F000E500B357F500B318E60033E8070133135D
:10A60000E50013D608013355C80293960801C182AC
:10A61000935703013377C802B385A6024207336814
:10A62000F700637AB80046989307F5FF6364180152
:10A630006367B8303E853308B8403357C8024203D9
:10A64000135303013378C802B386E6024208336825
:10A650006800637BD80046989307F7FF636518018D
:10A6600079176363D8003E874205598D8145828002
:10A6700001E60547B358C702416763EAE80EB7072A
:10A68000000163ECF82893D68801E1471787FFFFA4
:10A6900013078725369783460700BE969307000267
:10A6A000958FE5EB939E08013387154113DF080171
:10A6B00093DE0E018545935703013355E703337746
:10A6C000E703B306D5034207D98F63FAD700C697CD
:10A6D0001307F5FF63E4170163E6D7263A85958FE4
:10A6E00033D7E703420313530301B3F7E703B30E72
:10A6F000D703C207B3E7670063FBD701C69793068A
:10A70000F7FF63E51701791763E3D7013687420541
:10A71000598D828063E2D504C16763E2F604B7070E
:10A72000000163E4F61E13D7860161489787FFFF97
:10A730009387871BBA9703C70700130E000242973F
:10A74000330EEE40631A0E0C63EDB61C3335C500B4
:10A75000134515008145828081450145828093071C
:10A76000F00F63F3D71C13D786002148C1B7130736
:10A77000F00FC686E37C17F193D68800A14739B75E
:10A780001307F00FB286E378C7E493568600A1471B
:10A7900099B5B398F80033D6D50013DF0801335EBE
:10A7A000E6033397F500B356D500558F939E080105
:10A7B00093DE0E013313F50093550701B376E603DC
:10A7C000B387CE03C206CD8E63FBF600C696130692
:10A7D000FEFF63E4161763F2F616791EC6969D8E89
:10A7E00033D6E60393170701C183B3F6E603338537
:10A7F000CE02139706015D8F637BA70046979307F0
:10A80000F6FF636817136376A712791646979315B8
:10A810000E01098FD18D45B5B357E600B396C60139
:10A82000DD8E33D3E50013DF0601B357E303939EB8
:10A83000060193DE0E013398C5013357E5003368F6
:10A840000701935808013316C6013373E303B38538
:10A85000FE024203B368130163FBB800B698138786
:10A86000F7FF63EAD80C63F8B80CF917B698B38809
:10A87000B84033D7E803420813580801B3F8E80397
:10A880003383EE02C208B3E5080163FB6500B695A9
:10A890001308F7FF63EDD50863FB65087917B695D4
:10A8A000C207416FD98F1307FFFFB3F6E70093D8B4
:10A8B0000701718F4182B38EE602B3856540B3868E
:10A8C000C60213D80E013387E802BA96C2963386C1
:10A8D000C80263F3E6007A9693D80601469663E2CF
:10A8E000C5026385C5003E858145828041677D172D
:10A8F000F98EC206B3FEEE003315C501F696E37479
:10A90000D5FE1385F7FF8145828013D706014148A4
:10A9100031BD93560601C1477DB993D60801C147A1
:10A92000B5B38145054582803687014801B5428728
:10A9300085BF3E86E9BDBA871DBF328E4DB57915FC
:10A940004698D5B97915C69759BBB3C7A5008D8B65
:10A950003307C50081E78D4763EEC700AA876370A0
:10A96000E50A83C6050085078505A38FD7FEE3EAC0
:10A97000E7FE828093763500AA8791CA83C60500D8
:10A9800085078505A38FD7FE93F63700FDB793762D
:10A99000C7FF138606FE63F0C70683A3050083A2E4
:10A9A000450083AF850003AFC50083AE050103AE4C
:10A9B000450103A3850183A8C5019385450223A012
:10A9C000770003A8C5FF23A2570023A4F70123A6FD
:10A9D000E70123A8D70123AAC70123AC670023AE50
:10A9E00017019387470223AE07FF75B79041910780
:10A9F000910523AEC7FEE3EBD7FEE3E4E7F68280E2
:10AA00003D432A876373C3029377F700BDEFADE53B
:10AA1000937606FF3D8ABA960CC34CC30CC74CC74D
:10AA20004107E36BD7FE11E28280B306C3408A067A
:10AA30009702000096966780A6002307B700A3063A
:10AA4000B7002306B700A305B7002305B700A3048A
:10AA5000B7002304B700A303B7002303B700A30282
:10AA6000B7002302B700A301B7002301B700A3007A
:10AA7000B7002300B700828093F5F50F9396850009
:10AA8000D58D93960501D58D61B7939627009702D2
:10AA9000000096968682E78086FA9680C1171D8F01
:10AAA0003E96E374C3F8A5B735713ECBA6DA36C738
:10AAB0003AC942CD46CF9387418186DEA2DC8443EA
:10AAC00063DB05009307B0089CC07D55F6506654C3
:10AAD000D6540D61828093078020231AF1002AC486
:10AAE0002ACC814799C19387F5FF3EC83ECE7401B9
:10AAF000FD572E8426852C00231BF10036C2D92A4F
:10AB0000FD576355F5009307B0089CC061D0A2477C
:10AB10002380070065BF71713ED39307402006C7AD
:10AB20002EC632CD36CF3AD142D546D72312F102C6
:10AB30002ACC2AD4812897070000938707033EDE9A
:10AB4000FD57B2452313F102938741812ACE2AD6BD
:10AB5000884334092E862C0882C682D036CAE12961
:10AB6000BA404D6182800145828093F5F50F83479D
:10AB7000050091C76393B70082800505CDBF91C1E1
:10AB800001458280AA87850703C7F7FF6DFF3385DC
:10AB9000A7407D15828005C67D160147B307E500F5
:10ABA000B386E50083C7070083C606006396D70017
:10ABB0006304C7000507FDF33385D7408280014554
:10ABC0008280AA8709CA850503C7F5FF85077D1618
:10ABD000A38FE7FE65FB3E966393C70082808507DF
:10ABE000A38F07FED5BF01114AC803A9850022CC57
:10ABF00052C45AC006CE26CA4EC656C22E84328BC6
:10AC0000368A63EE260983D7C50013F7074851C774
:10AC100004408C495848AA8AB389B4408D44B3840F
:10AC2000E4020947B3C4E402138716004E9763F3A6
:10AC3000E400BA8493F70740D9C3A6855685EF1080
:10AC4000003D2A890DE5B14723A0FA008357C400CF
:10AC50007D5593E707042316F400F2406244D24482
:10AC60004249B249224A924A024B056182800C480D
:10AC70004E86EFF09FCD8357C40093F7F7B793E765
:10AC800007082316F4002328240144C84E99B384EE
:10AC900034412320240104C4528963732A01528958
:10ACA00008404A86DA85EF1020271C440145B38707
:10ACB00027411CC41C403E992320240179BF2686CD
:10ACC0005685EF10A0422A895DFD0C485685EF108D
:10ACD000402995BF83D7C500717126D34AD14ECF85
:10ACE00006D722D552CD56CB5AC95EC762C566C3B8
:10ACF00093F70708AA892E89B284B9C39C49A9E3AE
:10AD00009305000436C6EF1080302320A9002328C5
:10AD1000A900B24615E1B14723A0F9007D55BA500C
:10AD20002A549A540A59FA496A4ADA4A4A4BBA4B9F
:10AD30002A4C9A4C4D61828093070004232AF90023
:10AD400093070002A30CF1029307000302DA230D1C
:10AD5000F10236CE930B5002978AFFFF938ACAC83E
:10AD6000054C294B26848347040099C3639D7709CA
:10AD7000B30C9440638E0C00E6862686CA854E8509
:10AD8000EFF07FE6FD576304F51AD256E69636DA01
:10AD900083470400638D0718FD579304140002D005
:10ADA00002D63ED202D4A301010682DC83C5040090
:10ADB00015465685EF10A01413841400825731E510
:10ADC00013F7070109C713070002A301E10613F7F0
:10ADD000870009C71307B002A301E10683C6040078
:10ADE0001307A002638BE602B257268481462546EC
:10ADF0000347040093051400130707FD6374E60678
:10AE00008DC63ED61DA00504B9BF33055541331587
:10AE1000AC00C98F3ED0A28451BF72479306470051
:10AE2000184336CE634907023AD603470400930716
:10AE3000E002631FF704034714009307A002631B9B
:10AE4000F702F2470904138747009C433ACE63C1D7
:10AE500007023ED235A83307E04093E727003AD6F1
:10AE60003ED0E1B7B387670385462E84BA9749B7CA
:10AE7000FD57C5B7050402D28146814725460347E1
:10AE8000040093051400130707FD6378E606F1F24A
:10AE9000834504000D461785FFFF130565B5EF10C8
:10AEA000000611CD9787FFFF938787B41D8D930709
:10AEB0000004B397A700025505045D8D2AD0834591
:10AEC000040019461785FFFF1305C5B2930414004B
:10AED000230CB102EF10A00225C59757FFF7938707
:10AEE000671295E70257F2471377071009CF9107CA
:10AEF0003ECED257D2973EDAB5B5B38767038546C3
:10AF00002E84BA97ADBF9D07E19BA107D5B77808FE
:10AF100097060000938666CD4A860C104E859700F2
:10AF20000000E7000000FD572A8AE314F5FC835770
:10AF3000C9007D5593F70704E39307DE5255C5B367
:10AF4000780897060000938646CA4A860C104E85FC
:10AF50006D23D1BF411106C622C426C24AC0FD5787
:10AF6000639AF500FD54B24022442685024992447A
:10AF7000410182808357C60013F9F50F93F4F50F52
:10AF800093F7F7FD2316F6005C5A584285C71C5EFE
:10AF90003284635CF7001C401387F7FF18C0A38F4F
:10AFA00027FF5C4085075CC07DBFB285EF0030673E
:10AFB0007DD14DBF144A1C4281CE63FBF60083C68F
:10AFC000F7FF63979600FD1705071CC258C261BFC3
:10AFD0005CDE930746045CDA8D471CDE930766044B
:10AFE0001CC2854738C2230326055CC2ADBF411190
:10AFF00022C42E84CC5906C69DC1930744046384A1
:10B00000F500EF0010763C40232A04025CC081CB9F
:10B010005C5C01451CC0B2402244410182801C4856
:10B02000232204007D551CC08357C40093E7070208
:10B030002316F400CDB7130101D2970700009387C0
:10B04000A7F12326312D232CF1289309C10197075D
:10B050000000938707FA232C812C232A912C232884
:10B06000212D2324412D2322512D2320612D232EF8
:10B07000712B232C812B232E112C232A912B232857
:10B08000A12B2326B12BAA842E842324011223264C
:10B09000011223283113232EF12836CC130A500233
:10B0A000130BA002A54B2949978AFFFF938A4A9464
:10B0B000175CFFF7130C0CF58347060032C6638557
:10B0C0000732EF00B05E3246834D0600930C160047
:10B0D0006E9583471500A18BB1C35C406359F002A4
:10B0E000EF00D05C1C4003C707003A9503471500EA
:10B0F000218B19E36686C9B70327C11285071CC0D7
:10B1000005072326E11258407D1758C0F9B7832759
:10B11000C129A2852685829761D5E9BF639A4D171B
:10B1200023220112232E0110834716006397670123
:10B13000C147232EF110930C260083C50C00668DA9
:10B14000850C938705FD63F0FB060D465685EF00E1
:10B15000105B01CD330555418547B397A700032503
:10B16000C111668D5D8D232EA11083470D0013073D
:10B170007006930C1D006366F7081307500663F012
:10B18000E71C13077004636AF7021307500463F89F
:10B19000E71A638B0712638D470F8D47232AF1123D
:10B1A0002320211361A083274112B307F90293875B
:10B1B00007FDAE972322F11249B71307B005638349
:10B1C000E7126365F70213078005E398E7FC03279E
:10B1D000C11113670720232EE11041472320E112FC
:10B1E0001307E006B337F7008D073DA813073006B5
:10B1F0006387E71013074006E391E7FA2320211342
:10B20000C5B7130700076383E70C6365F7061307E9
:10B21000E006638FE70E6362F70C13079006E39E68
:10B22000E7F6232001128D47232AF1125C40635A6E
:10B23000F0108327C11193F7070481EFEF00104747
:10B240001C4003C707003A9503471500218B631282
:10B2500007108327411309476342F71234082286F7
:10B260006C0A2685352B85476300F5188947E3135B
:10B27000F5E881A813075007E382E7F81307800772
:10B28000E387E7F413073007E399E7F0894769BFDD
:10B290005C406352F0021C4003C707006316B715F9
:10B2A000850758401CC08327C1127D1758C08507E9
:10B2B0002326F11281B58327C129A285268582978D
:10B2C00079D90325811279ED7D55D5A00327C111C8
:10B2D00013670702232EE110DDBDA1472320F112E1
:10B2E000914799B7E6854E85EF0030008327C1115D
:10B2F000AA8C93E70704232EF110854735B78327DF
:10B30000C111232A011293E70704232EF11039BF3C
:10B310008327C11113F70701E31E07DC624793F58A
:10B3200017008326C1121306470091C532CC1C4377
:10B330002390D700C1B332CC1C4394C365BB95475F
:10B34000E5B58327C129A28526858297E30305EE0B
:10B350008DBF0327C11205072326E11258407D1730
:10B3600058C06355E00085071CC0C9BD8327C129AB
:10B37000A28526858297E30305ECA1B711476348B0
:10B38000F700340822866C0A26850123E9BDE30311
:10B390000CD6340822866C0A268597000000E70048
:10B3A0000000D1B58357C40093F7070491FF8320B1
:10B3B000C12D0324812D8324412D0329012D8329AF
:10B3C000C12C032A812C832A412C032B012C832B93
:10B3D000C12B032C812B832C412B032D012B832D7F
:10B3E000C12A1301012E828003258112C9B7797108
:10B3F00056CA9C49BA8A984522D426D24ECE52CCFF
:10B4000006D64AD05AC85EC6AA892E84B284368A25
:10B4100063D3E700BA879CC00347340419C3850788
:10B420009CC01C4093F7070281C79C4089079CC0C1
:10B430000329040013796900631A0900130B9401AE
:10B44000FD5B5C449840998F634CF9041C40834633
:10B45000340493F70702B336D000A5EB1306340487
:10B46000D2854E85829AFD576303F5041C40114630
:10B470009840998B544481446397C700B384E64055
:10B4800063D3040081441C4418486354F700998F27
:10B49000BE94014969047D5B63982405014509A8B0
:10B4A00085465A86D2854E85829A631E75017D55E2
:10B4B000B250225492540259F249624AD24A424B43
:10B4C000B24B456182800509ADBF3307D400130636
:10B4D0000003A301C7040347540493871600A297EF
:10B4E0008906A381E7049DBF85462286D2854E85C5
:10B4F000829AE30E65FB050945B7797122D426D2FD
:10B500004AD04ECE06D652CC56CA5AC8B68983C641
:10B5100085019307E0063289AA842E8413863504B8
:10B520006381F61E63E2D706930730066382F60A4C
:10B5300063EDD700638B061E930780056387F616BD
:10B54000930A24042301D40469A893074006638660
:10B55000F60093079006E395F6FE1C40084393F629
:10B56000070893054500C1C21C410CC363D80700FE
:10B570001307D002B307F040A301E4049776FFFF5E
:10B580009386C647294765A0930730076383F61A59
:10B5900063EFD7009307F006638FF6049307000765
:10B5A000E390F6FA9C4193E707029CC109A8930730
:10B5B00050076382F60493078007E393F6F8930736
:10B5C0008007A302F4049776FFFF93866644E5A004
:10B5D0001C43938A2504938647009C4314C323810C
:10B5E000F5048547BDA293F607041C410CC3BDDEDC
:10B5F000C207C187A5BF0C401C4313F8050813857B
:10B6000047006305080008C39C4339A093F505046F
:10B6100008C3FDD983D707001307F006638BE60C38
:10B620009776FFFF9386863D2947A30104044C408B
:10B630000CC463C5050008406D9908C099E3B28A3F
:10B6400091CDB28AB3F5E702FD1AB69583C5050020
:10B650002380BA00B3D5E70263F3E70AA147631E6C
:10B66000F7001C40858B91CB58401C4863C7E7000E
:10B6700093070003A38FFAFEFD1A3306564110C844
:10B680004E87CA867000A2852685EFF05FD67D5A68
:10B690006315450D7D55B250225492540259F2491A
:10B6A000624AD24A424B45618280A382D504977692
:10B6B000FFFF9386A6340C40084313F805081C418D
:10B6C00011056300080208C313F7150001C793E5CD
:10B6D00005020CC04147B1FB0C4093F5F5FD0CC0D1
:10B6E000A9B713F8050408C3E30008FEC207C18325
:10B6F000E1BF9776FFFF9386663021473DB7AE875F
:10B7000091B794411C43CC4913F8060813854700B0
:10B710006306080008C39C438CC301A808C393F6C2
:10B7200006049C43F5DA2390B70023280400B28A6C
:10B7300081BF1C43D04181459386470014C383AA2F
:10B7400007005685EF00A07B01C53305554148C071
:10B750005C401CC8A301040425B714485686CA855A
:10B7600026858299E30845F31C40898B8DE7B24713
:10B770004844E352F5F23E8539BF85465686CA8570
:10B7800026858299E30865F1050A5C443247998F62
:10B79000E345FAFEE9BF014A930A94017D5BF5B7E0
:10B7A0009C45011122CC26CA52C406CE4AC84EC6B8
:10B7B00056C25AC02A8A2E84B28491E7984D854792
:10B7C00011C3FD571CC41C40C18B99E79C421387D1
:10B7D000470098C283A907000149854A094B084CD4
:10B7E0001DC5631255099C4003C707005C48BA9702
:10B7F00083C7070089EF63180904F2406244D2440A
:10B800004249B249224A924A024B056182801C4059
:10B810000509C18B99E79C40850983C70700A38F61
:10B82000F9FE9840DC40050798C01844FD17DCC0BD
:10B830007D1718C409CBE344F0FA83270418A685C2
:10B840005285829749DD1C40C18B81EB5C448507A2
:10B850005CC41C4C99C3238009001C4801453E99D7
:10B860002328240159BF631B650189259C4083C798
:10B8700007003E9583471500A18BD1DBE31509FC3A
:10B88000084C8547E311F5FC8DBF5D719777FFFF8D
:10B890009387871ACAC03EC236899777FFFF93877E
:10B8A000E719944D3EC49777FFFF93876719A2C4A9
:10B8B0004EDE5AD86ECE3EC686C6A6C252DC56DAD8
:10B8C0005ED662D466D26AD08D47AA892E84B28DA4
:10B8D000170B0000130B8B536396F600170B000039
:10B8E000130BEB3D1C449306C015014A1386F7FF6A
:10B8F00063F7C600138A37EA9307D0151CC41C40AF
:10B900008566938606D09304C401D58F1CC0130CA2
:10B910004100A68A814B930C002083A70D000325CC
:10B920000C00094683C50700D92B25C185476390C4
:10B93000FB0E5C4099E71C40214758C093E7072065
:10B940001CC01C4093F7F7AF1CC01C441386F7FFC4
:10B9500010C485CF03A60D00138D1A00930716009F
:10B9600023A0FD00034606002380CA0003A64D0065
:10B97000EA8A7D1623A2CD006349C000032604187D
:10B98000EE854E850296631A0510850B8D47110CC6
:10B99000E395FBF85C4099E3A9475CC05C404848EC
:10B9A0009775FFFF938505099D8DFD7B056C568D71
:10B9B0002D2A814A930C0003938BFB6F130C0C8090
:10B9C00014441040C9C203A50D004C4803480500AB
:10B9D000C29583C50500A5C963189805B37586018E
:10B9E000A1C5850A63050A0085067D1A14C483A6CD
:10B9F0004D00FD1623A2DD006351D00483A60D0087
:10BA0000850623A0DD001444FD1614C455BF8947E4
:10BA1000E39DFBF21C4013F60760E31896F74147DD
:10BA200058C093E707100DB73376760110C08346F0
:10BA30000500050DA30FDDFE5DBF83260418EE850E
:10BA40004E85829669D1144093F6061085C263FC38
:10BA5000A4018345FDFF8326C417130AFDFF6E86EC
:10BA60004E858296528D0545630F9D041840418B8B
:10BA700021E723000D0054400146A6854E85029B18
:10BA800014400327090013F6060211CA9306470063
:10BA90002320D900184308C329A8814A6DB793F51C
:10BAA0001600130647009DCD2320C900184323101C
:10BAB000A7005844050758C41C48B3049D40D694B9
:10BAC000BE9404C80145B640264496440649F2593E
:10BAD000625AD25A425BB25B225C925C025DF24DCA
:10BAE000616182802320C90075B783C705001307F1
:10BAF000E0056388E7041387150081460146930536
:10BB000000103308C5002300D8000506E31BB6FE6D
:10BB10001306F7FF8DC793C616009308D0021308CB
:10BB2000D0053306F5002300D60083450700130631
:10BB30001700638415036384050191E93A86328511
:10BB400082801387250083C71500854645BFAE87D1
:10BB50003287C1BF9307D002E5BF83451700E38B4F
:10BB600005FFE3C9F5FE090785073306F500230045
:10BB7000D600E3CBB7FE55BF79714AD04ECE06D67C
:10BB800022D426D2AA892E899304190003C4F4FF73
:10BB90003A8536C632C42EC23AC031262295834732
:10BBA000150002479245A18B2246B246C9E793078A
:10BBB000D0026314F40883C70400054393042900EA
:10BBC000FDC641476392E60213070003639EE70048
:10BBD00083C704001307800593F7F70D6394E70C00
:10BBE00083C71400C1468904B708008063140300AA
:10BBF00093C8F8FF33FFD80201480145A54FE54E31
:10BC0000FD5233DED802138707FD63E4EF04BA87E1
:10BC100063DFD704630D58007D58636AAE00631478
:10BC2000AE006346FF0005483385A6023E958504B5
:10BC300083C7F4FFC9BF268981BF9307B00263059C
:10BC4000F400A2870143ADBF83C704009304290019
:10BC5000D5BF1387F7FB63E5EE00938797FC4DBFD5
:10BC60001387F7F963E5EE00938797FA55B7FD5709
:10BC7000631FF8009307200223A0F900468519EE00
:10BC8000B250225492540259F249456182806304B1
:10BC900003003305A0406DD6630408009385F4FFCC
:10BCA0000CC2F9BF93070003A1F2A14635BF1307E9
:10BCB0000003E38FE7F0A94605BF938741819C43CA
:10BCC000985309E71757FF17130787856FF0DFEAC7
:10BCD00079714AD04ECE06D622D426D2AA892E8990
:10BCE0009304190003C4F4FF3A8536C632C42EC249
:10BCF0003AC0552A22958347150002479245A18BE9
:10BD00002246B246BDEF9307D002631EF40683C7F6
:10BD10000400054393042900F5C241476392E602FB
:10BD200013070003639EE70083C704001307800521
:10BD300093F7F70D639FE70A83C71400C146890490
:10BD40007D57335ED70201480145254FE54EB37854
:10BD5000D702138707FD6364EF04BA8763D1D70660
:10BD6000634D08047D58636AAE006314AE0063C679
:10BD7000F80005483385A6023E95850483C7F4FF85
:10BD8000C9BF2689B1BF9307B0026305F400A2873B
:10BD9000014359B783C7040093042900D5BF138713
:10BDA000F7FB63E5EE00938797FC4DBF1387F7F928
:10BDB00063E7EE00938797FA55B77D587DBF635FC1
:10BDC00008009307200223A0F9007D5519EEB25018
:10BDD000225492540259F24945618280630403005F
:10BDE0003305A0406DD6630408009385F4FF0CC2B0
:10BDF000F9BF93070003A9F6A14699B713070003FB
:10BE0000E384E7F2A9462DBF938741819C43985371
:10BE100009E71747FF171307A7706FF07FEB0111B2
:10BE200022CC2E84CC5906CE26CA4AC84EC652C44D
:10BE3000930744046394F50493050040C92A11E96B
:10BE40007D55F2406244D2444249B249224A0561DA
:10BE50008280930700401CDC8347640448D81305A4
:10BE6000D53F2301F50083475404A300F500834721
:10BE700044042300F50008C00145E1B70329840309
:10BE8000931919004E869D24AA845DD9330A250191
:10BE9000AA854A865285EFE05FAB2320440144D84F
:10BEA000232C3403D1BF0325C50E828093874181A3
:10BEB0009C439C5389E79747FF179387676603A5C1
:10BEC000C70E828085E141116C00014511CA795588
:10BED00081CA834706009CC1034506003335A00094
:10BEE00041018280014519CA795589CA83470600F4
:10BEF0009CC1034506003335A0008280828093F503
:10BF0000F50F2A966314C50001458280834705001A
:10BF1000E38DB7FE0505FDB763F3A504B386C50041
:10BF2000637FD5029345F6FF8147FD176393F500C4
:10BF300082803387F600034807003387C7002A97BB
:10BF400023000701DDB73387F50083460700330779
:10BF5000F50085072300D700E317F6FE82808147AE
:10BF6000E5BFCDC583A7C5FF411122C406C626C2C1
:10BF70001384C5FF63D307003E94AA84292C9747F6
:10BF8000FF179387E7739C4389EF232204009747A9
:10BF9000FF1723A787722244B240268592444101AD
:10BFA000E5AA637EF40014403307D4006396E700EB
:10BFB0009843DC43369718C05CC0D1BFBA87D843DA
:10BFC00019C3E37DE4FE94433386D700631F8600E4
:10BFD0001040B29694C33386D700E31EC7FA1043CD
:10BFE0005843B29694C3D8C37DB76375C400B147B4
:10BFF0009CC055B71040B306C4006316D700144365
:10C000005843B29614C058C0C0C371B782800111A2
:10C0100026CA93843500F19806CE22CC4AC84EC673
:10C02000A104B14763F7F404B14463E6B4042A8978
:10C030009D229747FF179387A76898433A8431E476
:10C040009747FF17938707689C4381EB81454A8593
:10C05000D5289747FF1723A7A766A6854A85DD2021
:10C06000FD5963193507B1472320F9004A852D2270
:10C0700029A0E3DC04FAB1471CC10145F240624447
:10C08000D2444249B249056182801C40858F63C019
:10C090000704AD4663F6F6001CC03E9404C001A838
:10C0A0005C40631487021747FF17232BF7604A850C
:10C0B000E5201305B4009307440061993307F54068
:10C0C00055DF3A94898F1CC055BF5CC3CDB722871A
:10C0D0004040B5B7130435007198E30185FCB30502
:10C0E000A4404A858520E31B35FBB5BF81E5B285B9
:10C0F0006FF0FFF1011122CC06CE26CA4AC84EC607
:10C10000328401EEEFF0FFE50149F24062444A85D6
:10C11000D2444249B24905618280AE84AA89B528D9
:10C120002689E37485FEA2854E85EFF05FEE2A89AD
:10C1300069DDA6852286EFE05F81A6854E85EFF05A
:10C140005FE2E1B7411122C42A842E859767FF1769
:10C1500023A6078206C6EF603FA7FD576319F500C7
:10C160009767FF17938787819C4391C31CC0B24098
:10C1700022444101828091CD9307F00F63F7C700FD
:10C180009307A0081CC17D5582802380C50005450A
:10C190008280014582808280828083A7C5FF1385CB
:0EC1A000C7FF63D50700AA959C413E9582809B
:04C1B0000000030088
:08C1B4004000800000000000C3
:04C1BC000302010277
:04C1C0000403090467
:10C1C4000902430002010080320904000001020256
:10C1D40001000524001001052401000104240202C9
:10C1E40005240600010705820308000A090401006A
:10C1F400020A00000007050302400000070581024F
:10C2040040000000FF000000FE5000083851000804
:10C21400E85100089651000864510008000000002D
:10C22400000000000000000000000000000000000A
:10C2340000000000000000000000000000000000FA
:10C2440000000000000000000000000000000000EA
:10C2540000000000000000000000000000000000DA
:10C6340000000000000000000000000000030008EB
:10C6440000000020000000001403000800000000A7
:10C654000000000000000000000000002421000889
:10C6640034210008442100085C21000870210008DE
:10C674008421000890210008A02100080000000087
:10C68400602A0008802A0008402A000800000000F0
:10C694000000000000000000000000000000000096
:10C6A4000000000000000000000000000000000086
:10C6B4000000000000000000000000000000000076
:10C6C4000000000000000000000000000000000066
:10C6D4000000000000000000000000004300000013
:10C6E4000000000000000000000000000000000046
:10C6F40000000000000000000000000043000000F3
:10C704000000000000000000000000000000000025
:10C7140000000000000000000000000043000000D2
:10C724000000000000000000000000000000000005
:10C7340000000000000000000000000043000000B2
:10C7440000000000000000000000000000000000E5
:10C754000000000000000000000000004300000092
:10C7640000000000000000000000000000000000C5
:10C774000000000000000000000000004300000072
:10C7840000000000000000000000000000000000A5
:10C794000000000000000000000000004300000052
:10C7A4000000000000000000000000000000000085
:10C7B40000000000000000000000000076C1000836
:10C7C400C4BE000800000000B02A0008AC2A00081B
:10C7D400C0250008C0250008C0250008C0250008A1
:10C7E400C0250008C0250008C0250008C025000891
:10C7F400C0250008FFFFFFFFFFFFFFFFFFFFFFFF54
:10C80400FFFF0000010041534349490000000000BC
:10C814000000000000000000000000000000000014
:10C82400000000000000415343494900000000009B
:10C8340000000000000000000000000000000000F4
:10C84400000000000000000080190020FF0000002C
:10C8540000C201000000080001010000BC04002027
:08C864000000000001020304C2
:040000050800015C92
:00000001FF
